:020000040800F2
:10000000D809002035020008A14200088D380008F8
:10001000F13E0008251400082144000800000000FB
:100020000000000000000000000000005143000834
:10003000291400080000000011430008A94300082B
:100040004F0200084F0200084F0200084F0200084C
:100050004F0200084F0200084F0200084F0200083C
:100060004F0200084F0200084F0200084F0200082C
:100070004F0200084F0200084F0200084F0200081C
:100080004F0200084F0200084F0200084F0200080C
:100090004F0200084F0200084F0200084F020008FC
:1000A0004F0200084F0200084F0200084F020008EC
:1000B0004F0200084F0200084F0200084F020008DC
:1000C0004F0200084F0200084F0200084F020008CC
:1000D0004F0200084F0200084F0200084F020008BC
:1000E0004F0200084F0200084F02000800F002F81B
:1000F00000F090F80AA090E8000C82448344AAF132
:100100000107DA4501D100F085F8AFF2090EBAE82F
:100110000F0013F0010F18BFFB1A43F0010318473B
:100120002872000048720000103A24BF78C878C1D5
:10013000FAD8520724BF30C830C144BF04680C60ED
:10014000704700000023002400250026103A28BF35
:1001500078C1FBD8520728BF30C148BF0B60704739
:100160006E2900F09B81702900F0DD82662906F07F
:10017000F482652906F0F182672906F0EE82612992
:1001800006F0ED8203681B0A28BF41F0800169294F
:1001900000F04881642900F04581752900F0428112
:1001A0006F2900F06B82782900F0A982E92900F01C
:1001B0000582E42900F00282F52900F0FF81EF2991
:1001C00000F06882F82900F0A8820368DB0928BFE4
:1001D00041F08001632900F0A987732900F0AE8700
:1001E000E32900F0B987F32900F0BE8700207047AB
:1001F0001FB501F00FF804000020002105F08AF976
:10020000401C60600020002105F06EF9E0601FBD19
:1002100010B510BD00F0D0FF1146FFF7E9FF04F064
:100220006BFA01F0ADF803B4FFF7F2FF03BC01F085
:10023000F1F800000948804709480047FEE7FEE75B
:10024000FEE7FEE7FEE7FEE7FEE7FEE7FEE7FEE786
:1002500004480549054A064B704700001D44000844
:10026000ED000008D8030020D8090020D8050020A0
:10027000D805002000487047100000200FB41CB5BE
:10028000084B06AA7B4469460090059800F01FF9C8
:1002900004460020694600F02DF920461CBC5DF89C
:1002A00014FB00006D0200004FF000020429C0F0B2
:1002B000128010F0030C00F01B80CCF1040CBCF198
:1002C000020F18BF00F8012BA8BF20F8022BA1EBEA
:1002D0000C0100F00DB85FEAC17C24BF00F8012BCF
:1002E00000F8012B48BF00F8012B70474FF00002C7
:1002F00000B5134694469646203922BFA0E80C501C
:10030000A0E80C50B1F12001BFF4F7AF090728BFF6
:10031000A0E80C5048BF0CC05DF804EB890028BF72
:1003200040F8042B08BF704748BF20F8022B11F09B
:10033000804F18BF00F8012B704770477047704717
:10034000004870471000002010B5FFF793FF0068C9
:1003500010BD10B50446FFF78DFF046010BD70B5E9
:10036000044685690068C10601D5302600E02026D4
:10037000C00707D070BDD4E9012130469047206AFC
:10038000401C20626D1EF6D570BD70B504468569AF
:100390000078C00707D170BDD4E901212020904723
:1003A000206A401C20626D1EF6D570BD09684A05A2
:1003B00001D540B27047C905FCD500B27047096845
:1003C0004A0501D5C0B27047C905FCD580B2704757
:1003D00070B50C460546012A05D02878800600D560
:1003E000EA69002302E0012305E05B1C934202D28C
:1003F000E05C0028F9D1A869E618C01AA861286A4B
:10040000184428622846FFF7AAFF04E0D5E9012135
:1004100014F8010B9047B442F8D32846FFF7B5FF14
:1004200070BD00002DE9F0410646002410687529D2
:10043000314616A510D0FFF7B9FF002802DA404276
:1004400013A507E031688A0701D512A502E0490724
:1004500004D511A5012401E0FFF7B1FF00210A2214
:1004600006F1240709E0B0FBF2FCB0FBF2F302FB5B
:100470001C00303078541846491C0028F3D123461C
:100480002A463046BDE8F04100F061BA00000000A5
:100490002D0000002B000000200000001168026801
:1004A000006A530501D508700AE0D30501D508801C
:1004B00006E0130603D5C217C1E9000200E0086098
:1004C0000120704701694A1C02610878704700B535
:1004D0008FB0CDE901310021059105497944CDE97D
:1004E00003101146684600F029F90FB000BD000066
:1004F000E5FFFFFF0A6802F8010B0A607047000081
:100500002DE9FF5F15468A460446DFF8AC80F844C3
:100510000027D8E900103E46CDE9001010E03AF877
:1005200016106A4602A800F023FE411C07D021786D
:10053000890603D5E269391891420DD80744761C23
:100540002078800602D5E069B84205DDAE42E6DBE0
:100550003AF816000028E2D1A069C01BA06120462D
:10056000FFF7FDFED8E90010CDE90010002017E0EC
:100570003AF818106A4602A800F0FAFDB0F1FF3F01
:1005800081460BD000250DF1080B05E0D4E90121CF
:100590001BF8050090476D1C4D45F7D308F101008D
:1005A000B0428046E4DB206A384420622046FFF7F0
:1005B000ECFEBDE8FF9F0000326300002DE9F04132
:1005C0008046D21D22F007020025D2E90002F5295B
:1005D00015A614D0011E72F1000106DA0023D0EB3B
:1005E000030063EB020211A608E0D8F800108B07A5
:1005F00001D50FA602E0490701D50EA60125114637
:10060000002408F1240704E000F05CF930323A5588
:10061000641C50EA0102F7D12B463246214640467F
:10062000BDE8F04100F093B9000000002D0000008B
:100630002B0000002000000030B4002100F1240451
:1006400008E002F00705D208303542EA4372DB08C1
:100650006554491C52EA0305F3D10468002310A233
:10066000250708D504F020040C4304D0C4690123F5
:100670000CA2641EC46130BC00F069B910B5044618
:1006800021461068FFF79BFE02462046BDE8104059
:100690000023D1E7D21D22F00701D1E90023CBE7E7
:1006A0000000000030000000F0B40D46018809058C
:1006B00002D5214C7C4402E01F4C7C440E340021C6
:1006C00000F1240608E002F00F071209E75D42EA94
:1006D00003721B097754491C52EA0307F3D10278CD
:1006E0000023120704D5702D06D009B1022311345E
:1006F0002246F0BC00F02BB901231034F8E770B5A6
:1007000004460D4621461068FFF759FE0246294669
:100710002046BDE870400023C6E7D21D22F0070343
:10072000D3E90023C0E70368126843F020030360A5
:100730000823C3610023B7E7946100002DE9F05F4F
:10074000894604464FF0000ADFF874B1FB44C0F854
:1007500020A02046E1688847002874D0252806D0CC
:10076000D4E901219047206A401C2062F1E700266D
:100770005F462046E16888472028054607DB312D83
:1007800005D2781910F8200C08B10643F1E7B0073C
:1007900001D526F00406C4F81CA00027C4F818A050
:1007A0002A2D09D0284604F0DBFC38B304EB870877
:1007B000303DC8F8185019E059F8041B204604EBE6
:1007C00087029161E1688847012F054618D1E069E9
:1007D000002820DA26F020061DE0D8F8180000EBEB
:1007E000800005EB40003038C8F818002046E1686A
:1007F0008847054604F0B4FC0028EED1012F0AD04A
:100800002E2D08D12046E16888477F1C0546022F1F
:1008100046F02006C4DBA069002803DA404246F017
:100820000106A061F00701D026F010066C2D0BD058
:10083000682D09D04C2D39D06A2D35D0742D35D086
:100840007A2D33D016E038E0E1682F4620468847FD
:10085000B842054609D16C2F26D04FF48060E1687C
:10086000064320468847054604E06C2F1AD04FF413
:10087000807006430DB3A5F14100192802D8203538
:1008800046F400664A462946204626604E46FFF753
:1008900067FC80B101280BD0F61D26F0070000F19F
:1008A000080956E74020E4E78020D8E70020D6E793
:1008B00006F104094DE7284652E7206ABDE8F09F9B
:1008C0002461000030B5B0F10A0271F100034FEA73
:1008D000900E4EEA817EB0EB0E0061EB91014FEA83
:1008E000101E4EEA017E10EB0E0041EB11114FEA93
:1008F000102E4EEA016E10EB0E0041EB11214FEA73
:10090000104E4EEA014E10EB0E0041EB1141401823
:1009100041F100014FEAD00040EA41704FEAD101B5
:100920004FEA810444EA907410EB800544EB010423
:100930006D1944EB0404521BA3414FF0000348BF60
:100940000A3200D530BD401C41F1000130BD2DE917
:10095000F0470D4699469246044600F12408016886
:10096000880604D5E06921F01001216000E0012033
:10097000A84201DD471B00E00027A1697A1902EBBC
:100980000900081AA0612078C00602D42046FFF7AB
:10099000E6FC002608E0D4E901211AF80600904799
:1009A000206A401C761C20624E45F4DB2078C0068D
:1009B0000AD52046FFF7D3FC06E0D4E90121302018
:1009C0009047206A401C2062381EA7F10107F4DC22
:1009D00007E0D4E9012118F805009047206A401C7F
:1009E0002062281EA5F10105F3DC2046FFF7CDFCAF
:1009F0002078000602D50220BDE8F0870120FBE741
:100A00002DE9FF4F0C461E464FF0FF378BB0D2E961
:100A10000001DDF860800A908A46C1F30A5505B9E5
:100A20003D46002108464FF00000BAF1000F00F4E7
:100A3000400005DA00EB80004FF4400101EA50006D
:100A40004FEA9059B9F1010F00DDB9460A9850EA12
:100A50004A000ED044F61050A5F2FF3545432F143E
:100A6000B8F1000F1ED07542291E1EDDC9F100022B
:100A70001CE0B8F1010F4FF0000001D0302103E07D
:100A8000F24305E02154401CB042FBDB304600221B
:100A9000002121540B99C1F80880C1E900200FB052
:100AA000BDE8F08FBD1B6D1CDEE74A4600DA6942E7
:100AB00006A800F0F3FB06AB93E8070003AB83E85E
:100AC000070050460A9903F09AFE8DE80700A0F54A
:100AD00000501F3800900398002D0ADD42F21F01DC
:100AE0004A460844002303A90390684604F004F929
:100AF00009E0A0F500504A461F38002303A90390DF
:100B0000684604F00EF98DE807000004000C03D0DD
:100B10004FF0FF30410800E01046B8F1000F03D05D
:100B20000022009215461EE0751E05D4FFF7CAFE8E
:100B3000303262556D1EF9D5B3460122084302D00A
:100B400000227F1C04E02078302801D100227F1E83
:100B5000002A099784D01DE0112D07DAFFF7B2FEB5
:100B6000303262556D1C50EA0102F5D1084302D0C3
:100B70000098C8B10EE00021681E05E0235C625CAD
:100B800063542254401E491C8142F7DBAB46A81B2C
:100B9000401E0990002004F80B000B98099AC0F839
:100BA0000880C0E9002B7AE711264FF0000857E7CC
:100BB0002DE9F04F88460446D21D22F0070191B07E
:100BC000D1E90001CDE90A0104F0E2F902460B98EF
:100BD000C00F01D02D2007E02068810701D52B2010
:100BE00002E0202101EAC000032A099001D0072A6F
:100BF00005DB03464146204600F010FB0BE1207860
:100C0000800601D5E06900E00620B8F1650F814655
:100C100006D0B8F1660F18D0B8F1670F70D131E087
:100C20000020B9F1110F009001DB112301E009F15F
:100C300001030AAA01A90CA8FFF7E2FEDDE90C7086
:100C4000002609F10105834647E001204B4600904C
:100C50004FF000470AAA01A90CA8FFF7D1FEDDE971
:100C60000DB00C995D46002610B909F101000D1870
:100C7000B9EB050003D4C0F1FF3609F10105A5EB7E
:100C800009002BE0B9F1010F01DA4FF00109002052
:100C9000B9F1110F0090484601DD112300E0034631
:100CA0000AAA01A90CA8FFF7ABFEDDE90C704D46BE
:100CB00000268346207800070AD4AB4500DA5D465B
:100CC00001A8012D04DD411911F8011C302907D0BC
:100CD0004F4502DA17F1040F04DA012082460FE0D3
:100CE0006D1EEEE7002F02DCED1B3E4403E0781C96
:100CF000A84200DD7D1CB81B00F1010A4FF000473F
:100D00002078000703D4AA4501DB4FF0FF3A002109
:100D1000B7F1004F0DF143088DF8431024D00220A5
:100D20002B23002F01DA7F422D230A21021EA0F17E
:100D3000010000DC5FB197FBF1FC97FBF1F201FBD6
:100D40001C7C17460CF1300C08F801CDEEE7A8F139
:100D5000010003702188090501D5452100E06521C6
:100D6000A0F1010800F8011C09980FA9A1EB0807E0
:100D7000FF1D00B10120411901EBEA70A16938445F
:100D8000081A401EA0612078C00602D42046FFF752
:100D9000E6FA099828B1D4E901219047206A401C5D
:100DA00020622078C00622D52046FFF7D8FA1EE040
:100DB000002E04DBB34502DD01A8805D00E0302099
:100DC000D4E901219047206A401C2062761CAAF1D8
:100DD00001005FEA000A0AD100F01CFAC06801684D
:100DE000405CD4E901219047206A401C2062281E03
:100DF000A5F10105DCDC07E0D4E9012118F8010BBD
:100E00009047206A401C2062381EA7F10107F3DCDE
:100E10002046FFF7BAFA032011B041E62DE9F04F62
:100E200004460D46D21D22F0070089B0D0E9009794
:100E30004846394604F0ACF80246F80F01D02D239D
:100E400007E02068810701D52B2302E0202101EA79
:100E5000C0038DF820300BB1012000E00020032AF0
:100E6000824601D0072A04DB2946204600F0D6F945
:100E70003FE12078800601D40D2500E0E569C7F345
:100E80000A560D2D49DA00214FEA175B08464FF04C
:100E90000000002F00F4400007DA00EB80004FF460
:100EA000400100EBD07001EA60008115012901DDED
:100EB0004FF0FF3100224FEA850CBCF1180F06D32A
:100EC0001346ACF118004FF08052C24003E04FF4DB
:100ED000801323FA0CF30CF10C0CBCF1200F04D39B
:100EE000ACF1200C09FA0CF001E007FA0CF0002933
:100EF0004FF0004801DD18B90FE00ED140450CD38A
:100F000019EB02095F4121B9404502D19F4329EA0B
:100F10000209BBEB175F00D0761C2088000502D5C4
:100F20007B48784402E07A487844193808AA30238C
:100F300002F80A30037C0AF10101002E0AF1020ACC
:100F400053546A4602DC4FF0300101E04FF03101AA
:100F50004FF001088DF8001002D0A6F2FF3603E032
:100F600059EA470100D06B4E002D02DC21780907B9
:100F700004D54FF002082E218DF80110C44600213F
:100F80000BE0C7F303433F01C35C491C6D1E02F82D
:100F90000830052908F1010801DA002DF1DC0021F3
:100FA0000CE000EB1973491C1B786D1E082902F830
:100FB00008304FEA091908F1010801DA002DF0DCC8
:100FC00021688B0602D516E0A8F10108E04505DD91
:100FD00002EB080313F8013C302BF5D0B8F1000FF9
:100FE00009DD02EB080313F8013C2E2B03D109079E
:100FF00001D4A8F10108002D05DD3E2102F80810FA
:101000006D1E08F10108407C002E02F8080008F16E
:10101000010804DA2D20764202F8080002E02B20B5
:1010200002F808000A214FF47A70864208F101089C
:101030000BDB96FBF0F3303302F8083096FBF0F34D
:1010400008F1010800FB136601E0642E0CDB64204C
:1010500096FBF0F3303302F8083096FBF0F308F11A
:10106000010800FB136601E00A2E06DB96FBF1F097
:10107000303002F8080008F1010896FBF1F001FB9E
:101080001060303002F80800A16908F1010808EB8F
:10109000050202EB0A00081AA0612078C00602D4FB
:1010A0002046FFF75CF9216A08AE01EB0A002062D6
:1010B00004E0D4E9012116F8010B9047BAF1010AC6
:1010C000F7D22078C00602D52046FFF748F96E46D1
:1010D00009E016F8010B3E280FD0D4E90121904712
:1010E000206A401C2062B8F10108F2D22046FFF7C6
:1010F0004CF909B00320BDE8F08F206A2844206233
:1011000003E0D4E90121302090476D1EEBD3F8E7CE
:101110009559000002FCFFFF10B5436913B1AFF30E
:10112000008001E0FFF754F9012010BD127800F1B2
:1011300024010A7000224A700122EDE711684FF085
:10114000FF32E9E710B5436913B1AFF3008001E066
:10115000FFF7D6F9012010BD128800F12401828426
:101160000022C2840122EDE711684FF0FF32E9E767
:101170002DE9F04116460C46054600F043F8036899
:1011800093F80101012807D0FF2C12D8185D80B117
:1011900001202C70BDE8F081D3F8070132462146CA
:1011A00003F20713C7182846BC46BDE8F0410023E8
:1011B00060474FF0FF30EDE77546FFF7C1F8AE46E8
:1011C00005006946534620F00700854618B020B553
:1011D000FFF73EF8BDE820404FF000064FF0000753
:1011E0004FF000084FF0000BAC46ACE8C009ACE88B
:1011F000C009ACE8C009ACE8C00921F007018D4680
:101200007047000010B500F005F8001D10BD00BFCC
:101210000543000000487047300000202DE9F041F0
:101220001F46044603260168072A01F4006004DB18
:1012300008B116A505E016A503E008B115A500E064
:1012400015A521F010002060A069C01EA0610FB19B
:10125000401EA0612046FFF782F84FB1D4E901217A
:1012600038469047206A401C2062C01C206206E07D
:10127000206AFAE7D4E9012115F8010B9047761EA0
:10128000F8D22046FFF781F8BDE8F0814E414E00CC
:101290006E616E00494E4600696E66002DE9F047AA
:1012A000814616468AB0354878440DC88DE80D0051
:1012B00032487844801C03AC0DC884E80D0041F628
:1012C0009B300844372190FBF1F290FBF1F5A5F13A
:1012D000800501FB12041B3C02D56442012000E0A2
:1012E0000020DFF898A080460027FA44AAF1BE0A41
:1012F0000EE0E0070AD03246684607EB47010123BB
:101300000AEB810103F00DFD8DE8070064107F1CDE
:10131000002CEED1194F7F44AE3F19E0E80715D0FD
:1013200007EB04100DF1180A90E80E008AE80E0091
:10133000C068F04201D1981908903246012306A9ED
:1013400003A803F0EEFC03AB83E807006D10641CF8
:10135000002DE3D14FF0010332466946B8F1000F8A
:1013600003A802D003F0C8FC01E003F0DAFCC9E9ED
:101370000001C9F808200AB0BDE8F087A0560000B7
:1013800010B50446AFF300802046BDE81040FEF7DC
:101390004ABF00004FF0013C50F8042B51F8043BC9
:1013A0009A4221D1A2EB0C03934313EACC1317D139
:1013B00050F8042B51F8043B9A4215D1A2EB0C03D0
:1013C000934313EACC130BD150F8042B51F8043B90
:1013D0009A4209D1A2EB0C03934313EACC13DBD05E
:1013E0004FF00000704700BFD01A01BAB1FA81F186
:1013F00001F0180122FA01F0CB40DBB2C0B2C01AF2
:10140000C1F120012CFA01F3D11A914311EAC31161
:10141000E6D1704701491820ABBEFEE72600020066
:1014200070470000FFE7FEE77047000081B0EFF370
:10143000108072B60090FFE7FEE7000080B58CB028
:101440000B9040F21810C2F2000008904FF40071A7
:1014500000F004FA0898694600224A600A6047F2E0
:101460002E33C0F60003114600F056FE0B980078AC
:10147000C00790B1FFE740F21810C2F200000790D9
:1014800040F2D001C2F20001069100F0E3FA0699A1
:101490000798053100F0DEFA0CE040F2D000C2F20D
:1014A000000000F10A0140F21810C2F2000000F042
:1014B0004BFDFFE70B9800788008C00790B1FFE76D
:1014C00040F2D000C2F20000817CC27C037D407DEE
:1014D000EC46CCF8000040F21810C2F2000000F018
:1014E00093FDFFE70B9840684FF0864104F0BAFF88
:1014F00004F008FF03466846012141601E22026095
:1015000040F21810C2F200000590002103F014F818
:10151000059840F2D001C2F2000104911C3100F0A4
:1015200013FD04990598173100F094FA0B98007890
:10153000C008C007B0B1FFE740F2D000C2F200001F
:1015400090F8241090F8252090F8263090F8270085
:10155000EC46CCF8000040F21810C2F2000000F097
:1015600053FDFFE740F2D000C2F20000029000F10C
:101570002E0140F21810C2F20000039000F0E4FCCB
:1015800002990398293100F065FA0B980078000958
:10159000C007B0B1FFE740F2D000C2F2000090F8FF
:1015A000361090F8372090F8383090F83900EC4633
:1015B000CCF8000040F21810C2F2000000F024FD48
:1015C000FFE70B98806804F0B3FC02460B4647F235
:1015D0004131C0F600010DF12700FEF74FFE0B98D8
:1015E000806804F0A5FC4CF6CD42CCF6CC424CF61B
:1015F000CC43C3F6F07304F044FDE8B9FFE70B9861
:10160000806804F095FC4FF0663246F26663C3F6DC
:10161000EE7304F03DFD78B9FFE7694600204860AD
:10162000086040F21810C2F2000065210F220DF18F
:10163000270300F071FD0FE069460120486000209B
:10164000086040F21810C2F2000065210F220DF16F
:10165000270300F061FDFFE740F2D000C2F2000076
:1016600090F83B1090F83C2090F83D3090F83E0008
:10167000EC464FF0010ECCF804E0CCF8000040F24C
:101680001810C2F2000000F089FA0B9800784008A8
:10169000C007B0B1FFE740F2D000C2F2000090F8FE
:1016A0003F1090F8402090F8413090F84200EC460E
:1016B000CCF8000040F21810C2F2000000F0A4FCC8
:1016C000FFE740F21410C2F20000006838B1FFE7F3
:1016D00040F21810C2F2000000F00AFDFFE70CB063
:1016E00080BD000070B582B040F2D004C2F20004A8
:1016F0003A20A0721022E2722073182565734220EE
:10170000A0731421E1734FF0010E84F810E03C2027
:1017100020706270A070E57084F804E04120607170
:10172000A271E071257284F809E084F816E039208E
:10173000A0740F20E0744FF00C0C84F814C00B233D
:1017400063755626E67522766676A57684F81BE0E4
:101750004D2626776277A677E577552684F82060B0
:1017600084F8211084F822E084F828E04C2684F8DC
:10177000246084F8250084F826C084F827302626C3
:1017800084F8296084F82A2084F82B6084F82C508F
:1017900084F82DE02F2684F82E6084F82F2084F81A
:1017A000306084F83150272584F8325084F83310A3
:1017B00084F834E0252184F8361084F8370084F862
:1017C00038C084F83930092184F83B1084F83C2073
:1017D00084F83D30082084F83E0084F83FC04FF084
:1017E000130C84F840C04FF0060C84F841C04FF051
:1017F000030C84F842C0EC46CCF804E0CCF80000BE
:1018000040F21810C2F2000000F0C8F902B070BD3A
:1018100080B582B001903220009040F2D030C2F208
:101820000000006840F27001C2F200010968401A2D
:101830000099884210D9FFE740F2D030C2F2000090
:10184000006840F27001C2F2000108600198FFF7E1
:10185000F5FD02F075FFFFE702B080BD80B582B0F4
:1018600001900091019808B9FFE704E00198009900
:10187000FEF71AFDFFE702B080BD000080B584B01E
:1018800084460698CDF80CC08DF80B108DF80A2010
:101890008DF809308DF80800039808B9FFE7D7E004
:1018A0009DF809002028C0F2D380FFE79DF80900C9
:1018B000FF2800F3CD80FFE79DF80800C00738B986
:1018C000FFE701208DF8070000208DF8060006E0F4
:1018D00000208DF8070001208DF80600FFE79DF835
:1018E000090046F68E12C0F600020B2100FB012013
:1018F0004FF6A061CFF6FF71405C01308DF8050016
:101900009DF8050040F27801C2F200010870012044
:101910008DF80400FFE79DF804000A2800F3978083
:10192000FFE700208DF80300FFE79DF803009DF816
:101930000510884244DAFFE79DF809009DF804206D
:101940000B2100FB012046F68E11C0F60001084471
:101950004FF6A061CFF6FF71405C9DF80310C1F116
:101960000701C840C00790B1FFE703989DF80B102E
:101970009DF8032011449DF80A209DF804301A4474
:101980009DF80730C9B2D2B200F08EFA11E0039888
:101990009DF80B109DF8032011449DF80A209DF836
:1019A00004301A449DF80630C9B2D2B200F07CFA75
:1019B000FFE7FFE79DF8030001308DF80300B4E76F
:1019C0009DF8050007283BDCFFE79DF805008DF832
:1019D0000200FFE79DF80200082830DCFFE79DF8D1
:1019E0000800C00790B9FFE703989DF80B109DF819
:1019F000022011449DF80A209DF804301A449DF8F5
:101A00000630C9B2D2B200F04FFA11E003989DF847
:101A10000B109DF8022011449DF80A209DF8043017
:101A20001A449DF80730C9B2D2B200F03DFAFFE780
:101A3000FFE79DF8020001308DF80200CAE7FFE7DA
:101A4000FFE79DF8040001308DF8040063E7FFE72D
:101A500004B080BD80B58CB00B900A910B9818B182
:101A6000FFE70A9808B9FFE796E00A9800788DF832
:101A700027000A9840788DF826000A9880788DF81B
:101A800025000A98C0788DF824000A9800798DF80E
:101A900023009DF825009DF82710884207DBFFE70B
:101AA0009DF825009DF82710401A019006E09DF84A
:101AB00027009DF82510401A0190FFE70198079034
:101AC0009DF824009DF82610884207DBFFE79DF86B
:101AD00024009DF82610401A009006E09DF826008C
:101AE0009DF82410401A0090FFE7009806909DF89A
:101AF00027109DF825204FF0FF3091420146B8BFD6
:101B0000012105919DF826109DF824209142B8BF2F
:101B10000120049007980699401A0390FFE70B985C
:101B20009DF827109DF826209DF8233000F0BCF981
:101B30009DF827009DF82510884208D1FFE79DF801
:101B400026009DF82410884201D1FFE724E0039885
:101B50000044029002980699494288420BDDFFE753
:101B600006990398401A039005999DF827000844A8
:101B70008DF82700FFE70298079988420BDAFFE704
:101B8000079903980844039004999DF82600084497
:101B90008DF82600FFE7C2E70CB080BD10B58AB013
:101BA0008C4686460D980C99CDF824E08DF823C01C
:101BB0008DF822208DF821308DF820108DF81F002F
:101BC0009DF821009DF82010884204DAFFE79DF877
:101BD0002100069003E09DF820000690FFE706989C
:101BE000C11700EB917080088DF81E0009989DF8D0
:101BF00023109DF8212011449DF81E30C91A9DF82C
:101C000022201A449DF81FC0EE46CEF808C04FF4BB
:101C1000B47CCEF804C04FF4877CCDF80CC0CEF86D
:101C200000C0D2B2C9B202F0FDFBDDF80CC00998C9
:101C30009DF823109DF81E3019449DF822201A4467
:101C40009DF81F40EE46CEF80840CEF804C04FF095
:101C5000B40CCDF810C0CEF800C0C9B2D2B202F0B8
:101C6000E1FBDDF810C009989DF823109DF81E30A7
:101C700019449DF822209DF820E07244D21A9DF864
:101C80001F40EE46CEF80840CEF804C04FF05A0C84
:101C9000CDF814C0CEF800C0C9B2D2B202F0C2FB77
:101CA000DDF814C009989DF823109DF821201144F7
:101CB0009DF81E30C91A9DF822209DF820E072443C
:101CC000D21A9DF81F40EE46CEF80840CEF804C068
:101CD0004FF0000CCEF800C0C9B2D2B202F0A2FBA5
:101CE00009989DF823309DF81EC003EB0C019DF868
:101CF00022209DF821E07344A3EB0C03023B9DF8E6
:101D00001FE0EC46CCF804E0CCF80020C9B2DBB20E
:101D100002F012FC09989DF823309DF822209DF8CE
:101D20001EC002EB0C019DF820E07244A2EB0C02F5
:101D30009DF81FE0EC46CCF804E0D2B2CCF80020CD
:101D4000CAB2194602F0F8FB09989DF823309DF8B5
:101D50001EC003EB0C0102319DF822209DF820E00B
:101D600072449DF821E07344A3EB0C039DF81FE03F
:101D7000EC46CCF804E0D2B2CCF80020C9B2DBB219
:101D800002F0DAFB09989DF823109DF821201144F8
:101D90009DF822309DF81EC003EB0C029DF820E058
:101DA0007344A3EB0C039DF81FE0EC46CCF804E071
:101DB000DBB2CCF80030D2B2CBB2194602F0BCFB99
:101DC00009989DF823109DF8212011449DF81E20AC
:101DD0008B1A991E9DF82220043BA2F1020C9DF85B
:101DE0001F40EE46CEF804405FFA8CFCCEF800C0EF
:101DF000C9B2DBB202F0A0FB09989DF823109DF850
:101E0000212011449DF81E208B1A991E9DF8222036
:101E1000043B02F1020C9DF81F40EE46CEF8044050
:101E20005FFA8CFCCEF800C0C9B2DBB202F084FBD2
:101E300009989DF823109DF81E208B18991C9DF879
:101E400022209DF820C062440433A2F1020C9DF8C8
:101E50001F40EE46CEF804405FFA8CFCCEF800C07E
:101E6000D2B2C9B2DBB202F067FB09989DF8231029
:101E70009DF81E208B18991C9DF822209DF820C0EB
:101E80006244043302F1020C9DF81F40EE46CEF886
:101E900004405FFA8CFCCEF800C0D2B2C9B2DBB20B
:101EA00002F04AFB0AB010BD83B002908DF8071013
:101EB0008DF806208DF80530029808B9FFE740E05C
:101EC0009DF807007F2810DCFFE79DF80700002839
:101ED0000BD4FFE79DF806001F2806DCFFE79DF8FE
:101EE0000600B0F1FF3F01DCFFE72AE09DF80700A4
:101EF0009DF8061001F0F80100EB0110ADF80200AA
:101F00009DF8050070B1FFE79DF8060000F007019D
:101F1000012000FA01F30299BDF80220885C184301
:101F200088540DE09DF8060000F00701012000FA3A
:101F300001F30299BDF80220885C98438854FFE7BA
:101F4000FFE703B07047000010B586B0059004911C
:101F5000049800788DF80F00049880788DF80E00B2
:101F6000049800798DF80D00049840788DF80C00E5
:101F70000498C0788DF80B00049840798DF80A0019
:101F8000049880798DF80900059818B1FFE7049846
:101F900008B9FFE736E005989DF80F109DF80C2072
:101FA0009DF80E309DF80BC09DF80940EE46CEF826
:101FB0000440CEF800C002F0BFFA05989DF80E105C
:101FC0009DF80B209DF80D309DF80AC09DF8094042
:101FD000EE46CEF80440CEF800C002F0ADFA059807
:101FE0009DF80D109DF80A209DF80F309DF80CC04B
:101FF0009DF80940EE46CEF80440CEF800C002F04D
:102000009BFAFFE706B010BD80B585B084460798FF
:10201000CDF810C0ADF80E10ADF80C20ADF80A30B8
:10202000ADF80800049808B9FFE75FE0BDF80E00BE
:10203000BDF80A100844802813DCFFE7BDF80E0045
:1020400000280ED4FFE7BDF80C00BDF808100844C6
:10205000202806DCFFE7BDF80C00B0F1FF3F01DCF3
:10206000FFE743E0BDF80E00ADF80600FFE7BDF85E
:102070000600BDF80E10BDF80A201144884235DA7A
:10208000FFE7BDF80C00ADF80400FFE7BDF8040061
:10209000BDF80C10BDF80820114488421FDAFFE794
:1020A000BDF80600BDF804206FF0700101EA0211CE
:1020B0000844ADF80200BDF8040000F0070101205B
:1020C00000FA01F30499BDF80220885C5840885456
:1020D000FFE7BDF804000130ADF80400D6E7FFE7E4
:1020E000BDF806000130ADF80600C0E705B080BDC0
:1020F00080B582B00190019808B9FFE709E0019826
:102100006A461F21116000227F231146FFF77CFFE2
:10211000FFE702B080BD000010B586B08C46864651
:1021200009980899CDF814E08DF813C08DF81220A5
:1021300003938DF80B108DF80A00059818B1FFE78E
:10214000039808B9FFE724E0FFE70398007800B39D
:10215000FFE705989DF813109DF81220039B1B784C
:102160009DF80AC0EE46CEF800C0FFF787FB40F2AC
:102170007800C2F2000000789DF80B1008449DF82A
:102180001310084401388DF81300039801300390B0
:10219000DBE706B010BD000080B582B0009000986B
:1021A00020B9FFE700208DF807003EE00099C868DD
:1021B000486100990868898800F0C6FA0099097A90
:1021C00088422AD1FFE700990120C8600098806901
:1021D00028B9FFE700F0D0FA00998861FFE700F026
:1021E000CBFA009A11699269801A884214D3FFE7EA
:1021F00000990868898800F0A7FA0099097A88424E
:1022000004D1FFE701208DF807000EE000990020BF
:1022100088618DF8070008E003E000990020C8609D
:10222000FFE700208DF80700FFE79DF8070002B0E8
:1022300080BD000085B00390029101928DF80330BB
:10224000039818B1FFE7029820B9FFE701208DF845
:10225000130015E0029803990860019803994860FB
:102260009DF80300039908720398006920B9FFE7FD
:10227000039932200861FFE700208DF81300FFE783
:102280009DF8130005B070478DB00C900B910020A5
:102290000A90FFE70B980A99C840002800F0C18017
:1022A000FFE70B980A9A012191400840099009988C
:1022B000002800F0B280FFE70A9820F00300082110
:1022C000C4F20101405808900A9800F00300810010
:1022D0000F2000FA01F1089808400890089805902E
:1022E0000C9840F60001C4F20101884203D1FFE7D7
:1022F0000020049026E00C9840F60041C4F2010151
:10230000884203D1FFE70120039018E00C9841F2C6
:102310000001C4F20101884203D1FFE702200290CC
:102320000AE00C9941F20042C4F2010204209142F9
:1023300008BF03200290FFE702980390FFE703988D
:102340000490FFE7059804990A9A02F003029200AC
:102350009140884232D1FFE7099A40F20041C4F22D
:102360000101086890430860099A40F20441C4F2F0
:102370000101086890430860099A40F20C41C4F2D8
:102380000101086890430860099A40F20841C4F2CC
:1023900001010868904308600A9800F0030081007A
:1023A0000F2088400890089B0A9820F0030108221B
:1023B000C4F20102885898438850FFE70998FF2823
:1023C00003D8FFE70C98019003E00C9804300190CB
:1023D000FFE7019807900998FF2804D8FFE70A98BB
:1023E0008000009006E00A996FF01F0000EB81006A
:1023F0000090FFE70098069007980068069A0F2162
:102400009140884304219140084307990860099A44
:102410000C99C8689043C860FFE70A9801300A9099
:1024200038E70DB07047000090B00F900E9100207B
:102430000D900990FFE70E9800680D99C84000289C
:1024400000F07F81FFE70D99012088400C900E98E5
:1024500000680C9908400B900B980C99884240F04A
:102460006C81FFE70E9840680590002851D0FFE787
:10247000059801283AD0FFE7059802283FD0FFE7EA
:10248000059803285FD0FFE70598112832D0FFE7B1
:102490000598122838D0FFE705980021C1F21101F4
:1024A000884236D0FFE705980021C1F21201884228
:1024B0002FD0FFE705980021C1F22101884228D0E2
:1024C000FFE705980021C1F22201884221D0FFE7F1
:1024D00005980021C1F2310188421AD0FFE7059822
:1024E0000021C1F23201884213D02FE00E98C0685B
:1024F00009902CE00E98C0680430099027E00E98EF
:10250000C0680830099022E00E98C0680C3009902D
:102510001DE00E98806818B9FFE70420099011E0CB
:102520000E988068012806D1FFE7082009900C98D2
:102530000F99086105E0082009900C980F994861EF
:10254000FFE7FFE703E00020099000E0FFE70B98BA
:10255000FF2803D8FFE70F98049003E00F9804309A
:102560000490FFE7049808900B98FF2804D8FFE731
:102570000D988000039006E00D996FF01F0000EBAE
:1025800081000390FFE70398079008980068079A76
:102590000F219140884309999140084308990860A8
:1025A0000E98C079C006002840F1C680FFE7FFE71B
:1025B00041F21800C4F20200016841F0010101601B
:1025C000006800F0010006900698FFE70D9820F0E3
:1025D00003000821C4F2010140580A900D9800F050
:1025E000030081000F2000FA01F10A9888430A9045
:1025F0000F9840F60001C4F20101884203D1FFE7C1
:102600000020029026E00F9840F60041C4F201013C
:10261000884203D1FFE70120019018E00F9841F2B2
:102620000001C4F20101884203D1FFE702200090BB
:102630000AE00F9941F20042C4F2010204209142E3
:1026400008BF03200090FFE700980190FFE7019882
:102650000290FFE702980D9901F00301890000FA4A
:1026600001F10A9808430A900A980D9921F0030194
:102670000822C4F2010288500E988079C006002812
:1026800009D5FFE70B9A40F20841C4F2010108683E
:102690001043086008E00B9A40F20841C4F20101BF
:1026A000086890430860FFE70E988079800600284C
:1026B00009D5FFE70B9A40F20C41C4F2010108680A
:1026C0001043086008E00B9A40F20C41C4F201018B
:1026D000086890430860FFE70E988079800700281B
:1026E00009D5FFE70B9A40F20441C4F201010868E2
:1026F0001043086008E00B9A40F20441C4F2010163
:10270000086890430860FFE70E988079C00748B1D9
:10271000FFE70B9A40F20041C4F201010868104340
:10272000086008E00B9A40F20041C4F20101086819
:1027300090430860FFE7FFE7FFE70D9801300D9039
:1027400079E610B07047000082B00190ADF8021039
:1027500001988068BDF80210084204D0FFE701200C
:102760008DF8010003E000208DF80100FFE79DF8DF
:10277000010002B07047000040F2D030C2F2000009
:102780000068704780B582B00090009820B9FFE7DC
:1027900001208DF8070021E00099242081F83D00F8
:1027A00000980168086820F001000860009800F0B7
:1027B00073FA009900200864009981F83D0000999F
:1027C0000863009981F83E00FFE70099002081F836
:1027D0003C00FFE700208DF80700FFE79DF80700A9
:1027E00002B080BD80B58EB00C900C9820B9FFE788
:1027F00001208DF8370043E10C9890F83D0040B976
:10280000FFE70C99002081F83C000C9800F068FA72
:10281000FFE70C99242081F83D000C9801680868B6
:1028200020F0010008600C980168086840F400403E
:1028300008600C980168086820F40040086000F007
:102840006FFC0A900C98406848F2A061C0F2010148
:1028500088420BD8FFE70A9948F28042C0F21E0274
:102860000020914238BF012009900AE00A9940F601
:102870000012C0F23D020020914238BF01200990B1
:10288000FFE70998012804D1FFE701208DF8370000
:10289000F6E00A984DF68361C4F21B31A0FB0110EB
:1028A000800C0B900C980068406820F03F000B995A
:1028B00008430C99096848600C980068006A20F089
:1028C0003F0008900C98406848F2A061C0F20101F6
:1028D000884204D8FFE70B98013007900EE00B9870
:1028E0004FF49671484344F6D351C1F26201A0FB04
:1028F0000101012000EB91100790FFE7089807996C
:1029000008430C99096808620C980068C0694CF685
:10291000FF71884306900C98406848F2A061C0F2AD
:10292000010188421FD8FFE70A9801380C994968CD
:102930004900B0FBF1F001306FF31F30032803D8DA
:10294000FFE7042005900BE00A9801380C994968CC
:102950004900B0FBF1F001306FF31F300590FFE745
:10296000059804904CE00C98806868B9FFE70A98D5
:1029700001380C99496801EB4101B0FBF1F00130DD
:102980006FF31F3003900DE00A9801380C994968E5
:1029900019225143B0FBF1F00130042161F31F30E3
:1029A0000390FFE70398000518B9FFE701200290A4
:1029B00023E00C98806868B9FFE70A9801380C9901
:1029C000496801EB4101B0FBF1F001306FF31F30BA
:1029D00001900DE00A9801380C9949681922514379
:1029E000B0FBF1F00130042161F31F300190FFE7EB
:1029F000019840F400400290FFE702980490FFE73E
:102A00000698049908430C990968C8610C980068F5
:102A1000006820F0C0000C9B1968DA691B6A1A4331
:102A2000104308600C980068806848F2FF318843C2
:102A30000C9A1168D36812691A43104388600C9885
:102A40000068C06820F0FF000C9B19685A699B69F8
:102A50001A431043C8600C980168086840F00100F0
:102A600008600C99002008640C9A202182F83D101F
:102A70000C9908630C9981F83E008DF83700FFE748
:102A80009DF837000EB080BD10B588B084460C9814
:102A90000B98DDF828E0CDF818C0ADF81610ADF8A9
:102AA0001420ADF81230ADF81000FFF765FE03906A
:102AB000069890F83D00202840F0E680FFE7069851
:102AC00003996A4611600221C0F210010122192304
:102AD00001F004F820B1FFE702208DF81F00D7E0D5
:102AE000FFE7069890F83C00012804D1FFE7022098
:102AF0008DF81F00CCE00699012081F83C00FFE72B
:102B0000FFE7069800680068C00738B9FFE7069835
:102B10000168086840F001000860FFE70698016856
:102B2000086820F4006008600699212081F83D00C3
:102B30000699402081F83E000699002008640A9812
:102B400006994862BDF81000069948850698408DA0
:102B50000699088506990020CFF6FF70C86206988E
:102B6000BDF81610BDF81420BDF81230DDF830C0E5
:102B7000039CEE46CEF80440CEF800C000F0BAFE4A
:102B800020B1FFE701208DF81F0081E0FFE70698E4
:102B9000008D002849D0FFE706980C99039A01F0B0
:102BA000CBF880B1FFE70698006C042807D1FFE757
:102BB00006980168086840F400700860FFE701208B
:102BC0008DF81F0064E006980168406A007808618B
:102BD0000699486A013048620699088D01380885CF
:102BE0000699488D0138488506980068406900F0CC
:102BF00004010120B0EB910F16D1FFE70698008D7C
:102C000090B1FFE706980168406A0078086106996C
:102C1000486A013048620699088D0138088506998E
:102C2000488D01384885FFE7B1E706980C99039A6B
:102C300000F0FEFE80B1FFE70698006C042807D183
:102C4000FFE706980168086840F400700860FFE735
:102C500001208DF81F001BE006980168086840F409
:102C6000007008600699202081F83D000699002038
:102C700081F83E00FFE70699002081F83C00FFE75D
:102C800000208DF81F0003E002208DF81F00FFE7F1
:102C90009DF81F0008B010BD80B582B0019001986A
:102CA000006845F20041C4F20001884215D1FFE7F7
:102CB00041F21C01C4F20201086820F4001008600F
:102CC00040F60040C4F2010000904021FFF7DCFA1A
:102CD00000988021FFF7D8FAFFE702B080BD00001E
:102CE00080B588B00790002006900590049003906E
:102CF0000798006845F20041C4F2000188422CD1D7
:102D0000FFE7FFE741F21800C4F20200016841F05A
:102D100008010160006800F0080002900298FFE7D7
:102D2000C0200390122004900320069040F600403B
:102D3000C4F2010003A9FFF777FBFFE741F21C0093
:102D4000C4F20200016841F400110160006800F45F
:102D5000001001900198FFE7FFE708B080BD000078
:102D600040F20800C2F20000027840F2D031C2F214
:102D700000010868104408607047000080B542F206
:102D80000001C4F20201086840F01000086003204E
:102D900000F08CF80F2000F005F800F03BF8002060
:102DA00080BD000080B582B0009040F20000C2F209
:102DB0000000006840F20801C2F200010A784FF4F6
:102DC0007A71B1FBF2F1B0FBF1F000F057FD20B1E8
:102DD000FFE701208DF8070018E000980F280DD8B4
:102DE000FFE700994FF0FF30002200F045F800980F
:102DF00040F20C01C2F20001086003E001208DF8EE
:102E0000070003E000208DF80700FFE79DF80700AA
:102E100002B080BD83B0FFE741F21800C4F20200A7
:102E2000016841F001010160006800F001000290BA
:102E30000298FFE7FFE741F21C00C4F202000168BC
:102E400041F080510160006800F0805001900198CD
:102E5000FFE7FFE70421C4F2010108680090009831
:102E600020F0E0600090009840F000700090009822
:102E70000860FFE703B0704780B586B08DF8170093
:102E8000049103920020029001F0EEFB02909DF964
:102E90001700019002980499039A01F003FA014681
:102EA000019801F0E9FB06B080BD000080B582B05A
:102EB0000190019801F002FC02B080BD80B584B0A1
:102EC00002900191029820B9FFE701208DF80F00D0
:102ED0001BE1019842F20001C4F20201096801F00D
:102EE0000701884216D9FFE742F20000C4F202004F
:102EF000016821F00701019A11430160006800F0A8
:102F000007000199884204D0FFE701208DF80F00E7
:102F1000FBE0FFE702980078800700282AD5FFE74A
:102F2000029800784007002809D5FFE741F2040124
:102F3000C4F20201086840F4E0600860FFE702980C
:102F400000780007002809D5FFE741F20401C4F228
:102F50000201086840F460500860FFE741F2040194
:102F6000C4F20201086820F0F000029A926810434F
:102F70000860FFE702980078C007002860D0FFE7EC
:102F80000298406801280ED1FFE741F20000C4F228
:102F9000020000688003002804D4FFE701208DF8B8
:102FA0000F00B2E021E00298406802280ED1FFE74E
:102FB00041F20000C4F2020000688001002804D43D
:102FC000FFE701208DF80F009FE00DE041F20000C7
:102FD000C4F2020000688007002804D4FFE7012043
:102FE0008DF80F0091E0FFE7FFE741F20401C4F222
:102FF0000201086820F00300029A5268104308603A
:10300000FFF7BAFB0090FFE741F20400C4F20200B0
:10301000006800F00C0002994968B0EB810F0ED0F7
:10302000FFE7FFF7A9FB0099401A41F28931884276
:1030300004D3FFE703208DF80F0066E0E4E7FFE725
:10304000019842F20001C4F20201096801F007018F
:10305000884216D2FFE742F20000C4F20200016883
:1030600021F00701019A11430160006800F0070098
:103070000199884204D0FFE701208DF80F0044E059
:10308000FFE702980078400700280CD5FFE741F2DF
:103090000401C4F20201086820F4E060029AD268D8
:1030A00010430860FFE702980078000700280DD55C
:1030B000FFE741F20401C4F20201086820F4605005
:1030C000029A126940EAC2000860FFE700F03AF88D
:1030D00041F20401C4F202010968C9B20A0946F6C4
:1030E0006411C0F60001895CC84040F20001C2F2E0
:1030F0000001086040F20C00C2F200000068FFF717
:1031000051FE00208DF80F00FFE79DF80F0004B07E
:1031100080BD000040F20000C2F20000006870476D
:1031200080B5FFF7F7FF41F20401C4F2020109681C
:10313000C1F3022246F67411C0F60001895CC84052
:1031400080BD000086B0002005900490039002909E
:10315000019041F20400C4F2020000680590059855
:1031600000F00C000146009100283FD0FFE70098D6
:10317000042804D0FFE70098082806D037E041F281
:103180000020C0F27A00019037E00598C0F3834137
:1031900046F67C10C0F60000405C02909DF81600D8
:1031A000C007C0B1FFE741F20400C4F202000068AA
:1031B000C0F3404146F68C10C0F60000405C04901D
:1031C000029841F20021C0F27A0148430499B0FB11
:1031D000F1F0039007E0029840F60011C0F23D01C3
:1031E00048430390FFE70398019006E0FFE741F2B0
:1031F0000020C0F27A000190FFE7019806B0704706
:1032000080B586B00490049820B9FFE701208DF8BE
:1032100017002EE304980078C007002800F0AE8065
:10322000FFE741F20400C4F20200006800F00C0065
:10323000042813D0FFE741F20400C4F20200006842
:1032400000F00C0008281BD1FFE741F20400C4F293
:1032500002000068C003002812D5FFE741F2000019
:10326000C4F2020000688003002808D5FFE7049834
:10327000406820B9FFE701208DF81700F9E27CE0F3
:10328000FFE704984068B0F5803F09D1FFE741F2BD
:103290000001C4F20201086840F48030086032E0A6
:1032A0000498406868B9FFE741F20001C4F20201E6
:1032B000086820F480300860086820F480200860E6
:1032C00020E004984068B0F5A02F0DD1FFE741F24F
:1032D0000001C4F20201086840F480200860086818
:1032E00040F4803008600CE041F20001C4F20201B9
:1032F000086820F480300860086820F480200860A6
:10330000FFE7FFE7FFE7FFE704984068D0B1FFE77A
:10331000FFF732FA0390FFE741F20000C4F2020027
:103320000068800300280CD4FFE7FFF725FA039913
:10333000401A652804D3FFE703208DF8170098E2B0
:10334000EAE719E0FFF718FA0390FFE741F20000FF
:10335000C4F202000068800300280CD5FFE7FFF7E5
:103360000BFA0399401A652804D3FFE703208DF870
:1033700017007EE2EAE7FFE7FFE7FFE7049800783F
:103380008007002840F18D80FFE741F20400C4F27D
:103390000200006810F00C0F13D0FFE741F20400A8
:1033A000C4F20200006800F00C00082829D1FFE7F1
:1033B00041F20400C4F202000068C003002820D4D7
:1033C000FFE741F20000C4F2020000688007002815
:1033D00009D5FFE704980069012804D0FFE7012020
:1033E0008DF8170045E241F20001C4F202010868BD
:1033F00020F0F800049A526940EAC2000860FFE732
:103400004EE00498006958B3FFE70021C4F242215E
:1034100001200860FFF7B0F90390FFE741F20000D8
:10342000C4F202000068800700280CD4FFE7FFF711
:10343000A3F90399401A032804D3FFE703208DF86A
:10344000170016E2EAE741F20001C4F2020108683F
:1034500020F0F800049A526940EAC20008601EE0B9
:103460000021C4F2422100200860FFF785F9039093
:10347000FFE741F20000C4F2020000688007002864
:103480000CD5FFE7FFF778F90399401A032804D316
:10349000FFE703208DF81700EBE1EAE7FFE7FFE71E
:1034A000FFE7049800780007002848D5FFE7049854
:1034B000806918B3FFE740F28041C4F24221012045
:1034C0000860FFF759F90390FFE741F22400C4F2C6
:1034D00002000068800700280CD4FFE7FFF74CF9D2
:1034E0000399401A032804D3FFE703208DF817003F
:1034F000BFE1EAE7012000F00DFF1FE040F280414C
:10350000C4F2422100200860FFF736F90390FFE77C
:1035100041F22400C4F202000068800700280CD5A4
:10352000FFE7FFF729F90399401A032804D3FFE7BF
:1035300003208DF817009CE1EAE7FFE7FFE7049816
:1035400000784007002840F1D880FFE700208DF880
:10355000070041F21C00C4F202000068C00000280D
:1035600013D4FFE7FFE741F21C00C4F20200016838
:1035700041F080510160006800F080500090009898
:10358000FFE701208DF80700FFE747F20000C4F2D3
:1035900000000068C005002822D4FFE747F20001C0
:1035A000C4F20001086840F480700860FFF7E4F896
:1035B0000390FFE747F20000C4F200000068C00576
:1035C00000280CD4FFE7FFF7D7F80399401A6528C5
:1035D00004D3FFE703208DF817004AE1EAE7FFE78D
:1035E000FFE70498C068012809D1FFE741F22001F4
:1035F000C4F20201086840F00100086031E004985C
:10360000C06868B9FFE741F22001C4F2020108680E
:1036100020F001000860086820F0040008601FE046
:103620000498C06805280DD1FFE741F22001C4F2DB
:103630000201086840F004000860086840F00100DA
:1036400008600CE041F22001C4F20201086820F099
:1036500001000860086820F004000860FFE7FFE749
:10366000FFE7FFE70498C068E0B1FFE7FFF784F8E1
:103670000390FFE741F22000C4F2020000688007D7
:1036800000280ED4FFE7FFF777F80399401A41F2BC
:103690008931884204D3FFE703208DF81700E8E062
:1036A000E8E71BE0FFF768F80390FFE741F220002E
:1036B000C4F202000068800700280ED5FFE7FFF77C
:1036C0005BF80399401A41F28931884204D3FFE73D
:1036D00003208DF81700CCE0E8E7FFE79DF807002E
:1036E000012809D1FFE741F21C01C4F20201086878
:1036F00020F080500860FFE7FFE70498C0690028C9
:1037000000F0B380FFE741F20400C4F20200006859
:1037100000F00C00082800F08280FFE70498C069E0
:1037200002285CD1FFE76021C4F24221002008603A
:10373000FFF722F80390FFE741F20000C4F2020015
:103740000068800100280CD5FFE7FFF715F8039902
:10375000401A032804D3FFE703208DF8170088E000
:10376000EAE70498006AB0F5803F0CD1FFE741F228
:103770000401C4F20201086820F40030049A92683F
:1037800010430860FFE741F20401C4F20201086837
:1037900020F47410049B1A6A5B6A1A431043086091
:1037A0006021C4F2422101200860FEF7E5FF03908A
:1037B000FFE741F20000C4F2020000688001002827
:1037C0000CD4FFE7FEF7D8FF0399401A032804D36F
:1037D000FFE703208DF817004BE0EAE71EE06021C9
:1037E000C4F2422100200860FEF7C6FF0390FFE705
:1037F00041F20000C4F202000068800100280CD5EC
:10380000FFE7FEF7B9FF0399401A032804D3FFE747
:1038100003208DF817002CE0EAE7FFE724E0049886
:10382000C069012804D1FFE701208DF8170020E0CE
:1038300041F20400C4F2020000680290029800F411
:1038400080300499096A884208D1FFE7029800F4A1
:1038500070100499496A884204D0FFE701208DF86E
:10386000170006E0FFE7FFE7FFE700208DF81700ED
:10387000FFE79DF8170006B080BD000080B582B05C
:103880000190019800F066FD02B080BDFFE7FEE701
:1038900082B0009000980068406900F480610120C7
:1038A000B0EB912F1ED1FFE7009801686FF48060A4
:1038B0004861009900200863009A202182F83D1099
:1038C000009981F83E000099086C40F004000864FB
:1038D000FFE70099002081F83C00FFE701208DF808
:1038E000070003E000208DF80700FFE79DF80700C0
:1038F00002B0704780B586B0DDF824C0DDF820C086
:103900000490ADF80E10ADF80C20ADF80A30049814
:103910000168086840F4807008600498089B099961
:103920006A4611604FF00111002200F0D7F880B113
:10393000FFE7049800680068C005002805D5FFE788
:1039400004994FF400700864FFE703208DF8170016
:1039500069E0BDF80E0000F0FE00049909680861F6
:103960000498089A099B0221C0F2010100F03AF97B
:1039700020B1FFE701208DF8170054E0FFE7002099
:10398000019004980068406901900498006880697B
:1039900001900198FFE704980899099A00F0CCF982
:1039A00080B1FFE70498006C042807D1FFE7049872
:1039B0000168086840F400700860FFE701208DF896
:1039C000170030E0BDF80A00012806D1FFE79DF896
:1039D0000C0004990968086121E09DF80D00049924
:1039E0000968086104980899099A00F0A5F980B15E
:1039F000FFE70498006C042807D1FFE704980168EA
:103A0000086840F400700860FFE701208DF8170097
:103A100009E09DF80C00049909680861FFE700209F
:103A20008DF81700FFE79DF8170006B080BD000075
:103A300080B584B0029001910092FFE7029800687F
:103A4000406900F004010020B0EB910F3ED1FFE788
:103A50000298FFF71DFF20B1FFE701208DF80F004E
:103A600038E00198013080B3FFE7FEF785FE00994A
:103A7000401A0199884203D8FFE7019820BBFFE76D
:103A800002980068406900F004010020B0EB910F3B
:103A900019D1FFE7029900200863029A202182F8D9
:103AA0003D10029981F83E000299086C40F0200018
:103AB0000864FFE70299002081F83C00FFE701203D
:103AC0008DF80F0006E0FFE7FFE7B7E700208DF86D
:103AD0000F00FFE79DF80F0004B080BD80B588B0EF
:103AE000DDF828C0069005918DF813200393FFE7B9
:103AF0009DF8160001280CD1FFE706980068406980
:103B0000BDF814100840401AB0FA80F04009029045
:103B10000BE0069800688069BDF814100840401A50
:103B2000B0FA80F040090290FFE702989DF8131068
:103B300088424FD1FFE703980130002849D0FFE7C2
:103B4000FEF71AFE0A99401A0399884203D8FFE744
:103B50000398E8BBFFE79DF8160001280CD1FFE7AA
:103B6000069800684069BDF814100840401AB0FA81
:103B700080F0400901900BE0069800688069BDF86C
:103B800014100840401AB0FA80F040090190FFE795
:103B900001989DF81310884219D1FFE7069900207B
:103BA0000863069A202182F83D10069981F83E00AC
:103BB0000699086C40F020000864FFE70699002091
:103BC00081F83C00FFE701208DF81F0006E0FFE7C9
:103BD000FFE78DE700208DF81F00FFE79DF81F002D
:103BE00008B080BD80B588B006900591049203931B
:103BF000FFE79DF8160001280CD1FFE70698006842
:103C00004069BDF814100840401AB0FA80F040092D
:103C100002900BE0069800688069BDF81410084017
:103C2000401AB0FA80F040090290FFE7029800289D
:103C30007AD1FFE706980068406900F480610120AE
:103C4000B0EB912F24D1FFE706980168086840F493
:103C500000700860069801686FF4806048610699FA
:103C600000200863069A202182F83D10069981F809
:103C70003E000699086C40F004000864FFE70699CE
:103C8000002081F83C00FFE701208DF81F004FE085
:103C900004980130002846D0FFE7FEF76DFD039938
:103CA000401A0499884203D8FFE70498D0BBFFE785
:103CB0009DF8160001280CD1FFE7069800684069BE
:103CC000BDF814100840401AB0FA80F04009019085
:103CD0000BE0069800688069BDF814100840401A8F
:103CE000B0FA80F040090190FFE70198C8B9FFE7FA
:103CF000069900200863069A202182F83D10069953
:103D000081F83E000699086C40F020000864FFE747
:103D10000699002081F83C00FFE701208DF81F0084
:103D200006E0FFE7FFE764E700208DF81F00FFE7EC
:103D30009DF81F0008B080BD80B584B0029001914D
:103D40000092FFE7029800684069C1B20020B0EB22
:103D5000D11F3DD1FFE70298FFF79AFD20B1FFE7A1
:103D600001208DF80F0037E00198013078B3FFE7AC
:103D7000FEF702FD0099401A0199884203D8FFE737
:103D8000019818BBFFE7029800684069C1B20020A3
:103D9000B0EBD11F19D1FFE7029900200863029A06
:103DA000202182F83D10029981F83E000299086CAA
:103DB00040F020000864FFE70299002081F83C00F1
:103DC000FFE701208DF80F0006E0FFE7FFE7B9E706
:103DD00000208DF80F00FFE79DF80F0004B080BDB4
:103DE00080B58CB000200B900A9009900890FFE7F6
:103DF00041F21800C4F20200016841F010010160B4
:103E0000006800F0100007900798FFE7FFE741F215
:103E10001800C4F20200016841F02001016000684E
:103E200000F0200006900698FFE7FFE741F2180037
:103E3000C4F20200016841F004010160006800F072
:103E4000040005900598FFE7FFE741F21800C4F26F
:103E50000200016841F008010160006800F00800FC
:103E600004900498FFE7C02008900020019009907A
:103E7000012002900A9040F60000C4F2010008A957
:103E80000391FEF7D1FA019A0298039940F6034391
:103E9000089309920A9040F60040C4F20100FEF730
:103EA000C3FA0CB080BD000080B582B040F27C0047
:103EB000C2F20000019045F20041C4F2000101602D
:103EC00041F68021C0F20601416000218160C1609D
:103ED0004FF48042026141618161C1610162FEF77C
:103EE00081FC18B1FFE7FDF7A1FAFFE702B080BD42
:103EF000FFE7FEE780B584B0039003980C3040F6EE
:103F00000001C4F201010191402200230293FEF757
:103F100091F9029B0398283040F60041C4F2010158
:103F200000910222FEF786F90099029B0398443023
:103F30004FF48062FEF77EF90099029B039860308F
:103F40000122FEF777F90099029B03987C304FF429
:103F50000062FEF76FF90199029B03989830802266
:103F6000FEF768F903994620C861039988630399AD
:103F70004865039908670399C1F88C000399C1F853
:103F8000A80003994FF07E50886004B080BD000007
:103F900080B584B00390039840684FF07E5102F0E2
:103FA000A1F880B9FFE703990020486003980078E2
:103FB0004008C00730B9FFE70399087800F0FE0019
:103FC0000870FFE717E003984068002102F083F8CB
:103FD00080B9FFE7039800784008C00728B1FFE7E1
:103FE00003994FF07E50486003E003990020486039
:103FF000FFE7FFE7FFE740F20400C2F200000068BD
:104000000021C4F2C82102F02DFA01464FF07E5083
:1040100002F082F840F2CC31C2F20001086003984D
:104020000078C007D0B1FFE7039800780009C00707
:1040300098B9FFE703980078C008C00768B9FFE7A0
:104040000398816840F2CC30C2F200000290006810
:1040500002F008FA02990860FFE706E040F2CC316E
:10406000C2F2000100200860FFE703980078000911
:10407000C00720B3FFE703980078C008C007F0B975
:10408000FFE703984068002102F02CF8B0B9FFE781
:1040900040F20400C2F2000000680021C4F2C8210E
:1040A00002F0E0F901460020CBF6807002F034F80F
:1040B00040F2CC31C2F200010860FFE7FFE703984D
:1040C0000078C008C007F8B1FFE70398007800093E
:1040D000C007C8B9FFE740F20400C2F20000006860
:1040E0000021C4F2C82102F0BDF901464FF07E5014
:1040F00002F012F80146084601F046FF40F2CC31CA
:10410000C2F200010860FFE740F2D030C2F20000C6
:10411000006840F27401C2F200010968401A0B28DD
:1041200017D3FFE740F2D030C2F20000006840F23F
:104130007401C2F20001086040F2CC30C2F200000B
:10414000016803980190406801F01EFF01994860E2
:10415000FFE704B080BD000080B582B001900198F7
:104160000C30FEF719F870B1FFE70198006A48B902
:10417000FFE740F21411C2F20001086880F001006C
:104180000860FFE7FFE701982830FEF705F898B1CF
:10419000FFE70198C06B48B9FFE701990878012251
:1041A000824300F0FE0010440870FFE70199087890
:1041B00040F00400087005E00199087800F0FB0069
:1041C0000870FFE701984430FDF7E6FF30B1FFE7E4
:1041D0000199087840F00800087005E00199087816
:1041E00000F0F7000870FFE701986030FDF7D4FF9A
:1041F00030B1FFE70199087840F01000087005E041
:104200000199087800F0EF000870FFE701989830F6
:10421000FDF7C2FF88B1FFE70198D0F8AC0058B9AC
:10422000FFE701990878012222EA500200F0FD0020
:1042300040EA42000870FFE7FFE701987C30FDF795
:10424000ABFF58B3FFE70198D0F8900080B9FFE7C3
:1042500001980090806801F06BFE00220023C3F6F5
:10426000E07301F09FF901F06BF900998860FFE7B6
:104270000198806801F05CFE49F69A12C9F699121D
:1042800049F69913C3F6A97301F002FF28B9FFE7B5
:1042900001994FF07C508860FFE7FFE702B080BDD6
:1042A000FFE7FEE788B0079006910592079800F0B7
:1042B000070004900498C0F10700052803D3FFE726
:1042C0000420019004E00498C0F107000190FFE78A
:1042D0000198039004980430062803D8FFE70020D3
:1042E000009003E0049803380090FFE700980290E4
:1042F00006980399012202FA01F101390840029B54
:10430000984005999A40013A1140084308B0704717
:104310007047000082B00190019840F20001C2F2A3
:1043200000010968C90844F6D352C1F26202A1FB38
:104330000221890948430090FFE700BFFFE700988A
:10434000411E00910028F8D1FFE702B0704700003D
:104350007047000080B582B0009000980138B0F13D
:10436000807F03D3FFE70120019019E00098013816
:104370004EF21401CEF2000108604FF0FF300F2121
:1043800000F07AF94EF21801CEF200010020086028
:104390004EF21002CEF20002072111600190FFE7F9
:1043A000019802B080BD000080B5FEF7D9FC80BD49
:1043B00080B590B006A800902821FBF797FF0098E1
:1043C0000023059304930393029301930122069221
:1043D0004FF48031079108930A9202220D920E91B8
:1043E0004FF4E0110F91FEF70BFF18B1FFE7FDF757
:1043F0001DF8FFE70F200190022102910020039099
:104400004FF480620492059001A8FEF757FD18B1A1
:10441000FFE7FDF70BF8FFE710B080BD7047000025
:10442000FFE7FEE7B0B590B094468E460446169876
:104430001599149A0F948DF83BE08DF83AC08DF8D9
:104440003930ADF83620ADF834108DF83300002047
:104450000B900A90BDF836000990FFE70998BDF867
:104460003410884265DCFFE79DF83B0001F066FFF1
:1044700002909DF8390001F061FF0190099801F068
:10448000DBFA48F26E62CFF21B02039242F2F9139A
:10449000C4F20903049301F05FFB0022059248F285
:1044A0000003C4F26603069301F030F901F048F806
:1044B00000F05EFE0146019801F0D4FF029901F080
:1044C00063FD00F013FF01F01DFF0B909DF83A0013
:1044D00001F034FF08909DF8390001F02FFF07909C
:1044E000099801F0A9FA039A049B01F035FB059A9B
:1044F000069B01F00BF901F023F800F031FF0146B3
:10450000079801F0AFFF089901F03EFD00F0EEFEC4
:1045100001F0F8FE0A900F989DF82C109DF82820C5
:104520009DF83330FDF7C0FCFFE709980130099092
:1045300094E710B0B0BD000010B58CB08C46864634
:104540000F980E99CDF82CE08DF82BC08DF82A200D
:104550008DF829308DF828108DF827009DF8290056
:104560009DF82B10884207DBFFE79DF829009DF896
:104570002B10401A029006E09DF82B009DF82910A0
:10458000401A0290FFE7029808909DF828009DF8D5
:104590002A10884207DBFFE79DF828009DF82A10C3
:1045A000401A019006E09DF82A009DF82810401A54
:1045B0000190FFE7019807909DF82B109DF82920A6
:1045C0004FF0FF3091420146B8BF012106919DF89E
:1045D0002A109DF828209142B8BF01200590089824
:1045E0000799401A0490FFE70B989DF82B109DF84F
:1045F0002A209DF82730FDF757FC9DF82B009DF8E9
:104600002910884208D1FFE79DF82A009DF828105C
:10461000884201D1FFE724E0049800440390039806
:104620000799494288420BDDFFE707990498401A31
:10463000049006999DF82B0008448DF82B00FFE7A5
:104640000398089988420BDAFFE708990498084410
:10465000049005999DF82A0008448DF82A00FFE788
:10466000C2E70CB010BD00004EF60C50CEF20000B8
:104670000068C0F30220704782B08DF807000091F7
:104680009DF9070000280AD4FFE7009800019DF972
:1046900007104EF20042CEF2000288540BE0009860
:1046A00000019DF8071001F00F014EF61452CEF2F2
:1046B00000028854FFE702B07047000083B0029008
:1046C000029800F0070000904EF60C51CEF2000167
:1046D0000868019001984FF6FF0210400190019880
:1046E000009A40EA02200022C0F2FA5210430190E0
:1046F0000198086003B0704780B582B00020019037
:10470000FEF73CFBFFF754FEFFF76AFBFFF7CCFB1D
:1047100040F21830C2F20000FFF7ECFBFCF7E2FFBA
:10472000FFE740F21830C2F200000090FFF714FDDE
:104730000098FFF72DFC0098FDF76AF8F1E70000FC
:1047400080B586B000208DF81700FFE79DF81700B0
:1047500003283BDCFFE79DF81700B030C0B200F043
:1047600037F8002000F034F8102000F031F89DF800
:10477000171040F21810C2F2000000EBC110694699
:1047800064228A6080224A60086040F27C00C2F2A3
:104790000000782140220123FEF776F98DF81600FB
:1047A0009DF8160058B1FFE740F27C00C2F200000D
:1047B0000490FDF7E7FF0498FEF714F8FFE7FFE722
:1047C0009DF8170001308DF81700BFE706B080BDD7
:1047D00080B584B08DF80F0069464FF48070886012
:1047E00001234B600DF10F00086040F27C00C2F223
:1047F000000078210022FEF747F904B080BD5FEA8F
:10480000400C08BF91F0000F4FEA8C234FEAC12201
:1048100043EA51514FEA1C5018BF00F5F0404FEAEF
:10482000300018BF41F000415FEA6C5C00F0298065
:10483000BCF1FF3F08BF40F080407047130C06BF3B
:1048400012044FF0100C4FF0000C130E04BF1202B4
:104850000CF1080C130F04BF12010CF1040C930FA0
:1048600004BF92000CF1020CD30F04BF52000CF1F4
:10487000010C11464FF00002A0F11F00A0EB0C004C
:10488000704711F0004F08BF704731F000413FF40E
:10489000D5AF0B0C06BF09044FF0100C4FF0000C05
:1048A0000B0E04BF09020CF1080C0B0F04BF090129
:1048B0000CF1040C8B0F04BF89000CF1020CCB0F20
:1048C00004BF49000CF1010CCCF1200322FA03F3E0
:1048D00041EA030102FA0CF2A0EB0C0000F1010026
:1048E0007047000023F07F4720F07F4C80EA0300F0
:1048F00000F00040ACEB070303F57C5303F1FF032A
:104900002DE9804909B44FEA144324EA03484FEAE9
:10491000154B25EA0B4E0FF2042606EB13273E78C3
:1049200003FB0667C7F5000707FB06F64FEAD64606
:1049300006F102064FEA543707FB066CCCF1005C27
:104940004FEA1C472CEA074C0CFB06F507FB06F464
:1049500004EB15464FEA961649085FEA320234BF67
:1049600000204FF000404FEAD13706FB07FC4FEA2A
:104970001C4C0CFB0BF7D21B03FB0CF761EB070184
:104980000CFB0EF7B0EB074072EB17420CFB08F77D
:1049900034BFA2EB0742B2EB074261EB17414FEA8B
:1049A0000C444FEA910706FB07FC4FEA1C4C0CFB3A
:1049B0000BF7B0EBC74072EB573203FB0CF734BF79
:1049C000A2EBC742B2EBC74261EB57310CFB0EF7CB
:1049D000B0EBC70072EB57720CFB08F734BFA2EBC9
:1049E000C702B2EBC70261EB57714FEA816141EA3E
:1049F00092114FEA826242EA90124FEA806004EB21
:104A0000CC04039F4FEAD13706FB07FC4FEA1C4C4E
:104A10000CFB0BF7D21B03FB0CF761EB07010CFB44
:104A20000EF7B0EB074072EB17420CFB08F734BFF0
:104A3000A2EB0742B2EB074261EB17414FEA8C55FC
:104A400004EB9C244FEA910706FB07FC4FEA1C4C41
:104A50000CFB0BF7B0EBC74072EB573203FB0CF7C4
:104A600034BFA2EBC742B2EBC74261EB57310CFB3C
:104A70000EF7B0EBC70072EB57720CFB08F734BFB0
:104A8000A2EBC702B2EBC70261EB57714FEA81613B
:104A900041EA92114FEA826242EA90124FEA806044
:104AA00015EB4C2544F100044FEAD13706FB07FC17
:104AB0004FEA1C4C0CFB0BF7D21B03FB0CF761EB12
:104AC00007010CFB0EF7B0EB074072EB17420CFB33
:104AD00008F734BFA2EB0742B2EB074261EB174184
:104AE0004FEA813141EA92414FEA823242EA9042F2
:104AF0004FEA80304FEA0C7615EB1C1544F10004A8
:104B000048EA03434EEA0B484FF0000EB2EB080CA4
:104B100071EB030724BF624639464EEB0E0E4FF091
:104B2000000B0018524149414BEB0B0BB2EB080C48
:104B300071EB03077BF1000B24BF624639464EEB55
:104B40000E0E4FF0000B0018524149414BEB0B0B7E
:104B5000B2EB080C71EB03077BF1000B24BF62463C
:104B600039464EEB0E0E51EA020718BF46F0010619
:104B700016EB0E7655F1000254F1000103D5BDE8A5
:104B80008901BDE80088BDE88901BDE80048B61983
:104B9000524141EB0101A3F10103704780807F7E08
:104BA0007D7C7B7A797877767675747372717170A3
:104BB0006F6E6E6D6C6C6B6A6A6968686766666555
:104BC0006464636362616160605F5F5E5E5D5D5CE3
:104BD0005C5B5B5A5A595958585757565655555554
:104BE0005454535352525251515050504F4F4F4EB4
:104BF0004E4D4D4D4C4C4C4B4B4B4A4A4A49494902
:104C00004848484747474746464645454544444443
:104C10004443434343424242424141419C46002B6C
:104C200030D477002BD04FEA37071CB503B44FF0D0
:104C300010004FF01001BAF1000F06D0BCF1000FC8
:104C4000DCBF40F0080040F008014FF000000FBC4E
:104C5000BDE810400BF1010BBBF1010F08BF5FEA8B
:104C6000170722BF12F1010211F101014FF00041BB
:104C700043F1000300F0004043EA00007047F9D31D
:104C80005708D0E746EA06464FEA164613F1400FAA
:104C90001FDD13F1200FDFBF16430A46002120332A
:104CA0005B42BED0C3F1200746EA06464FEA1646ED
:104CB00002FA07F746EA070622FA03F2C3F12007D1
:104CC00001FA07F742EA070221FA03F14FF0000365
:104CD000A7E746EA020646EA06464FEA164646EACD
:104CE0000106BCBF46EA0646360C4FF000034FF003
:104CF00000024FF0000194E72DE9804C70B49A4611
:104D0000934691E8380007C831EA400C48BF34EABE
:104D1000430C03D5FFF7E6FDFFF780FFF0BCBDE8CD
:104D2000008C2DE9804C70B49A46934691E8380087
:104D300007C810F0804F08BF13F0804F03D100F078
:104D400005F8FFF76BFFF0BCBDE8008C20F07F4753
:104D500023F07F4C80EA030000F0004007EB0C03D7
:104D6000A3F57C53A3F1FE0392F0000F00F0B38093
:104D700095F0000F00F077802DE901494FEA1140CE
:104D800021EA00484FEA144624EA064700FB06FCE5
:104D900008FB06F607FB08F818EB06484CEB164C28
:104DA00000FB07F718EB07484CEB17404FEA124B94
:104DB00022EA0B4E4FEA154625EA06470BFB06FC96
:104DC0000EFB06F607FB0EFE1EEB064E4CEB164CDA
:104DD0000BFB07F71EEB074E4CEB174B18EB0B08C2
:104DE00040F1000018EB0E0B58EB000840F10000FA
:104DF0008F1A4FF000014FF000063CBFC943661BFD
:104E000014BFB5EB040C00213CBFC943F61B4FEAAD
:104E1000174427EA04454FEA1C472CEA074C04FBD9
:104E2000076205FB07F70CFB05F616EB074642EB9E
:104E3000174204FB0CFC16EB0C4642EB1C421BEB2E
:104E4000060658EB020241414EEA8E0E46EA9E06E5
:104E500001D5BDE80189B619524141EB0101A3F129
:104E60000103BDE801894FEA144524EA05464FEAEB
:104E7000114721EA074C05FB07F406FB07F70CFB7B
:104E800006F111EB074144EB174405FB0CFC11EB59
:104E90000C4144EB1C444FEA124722EA074C05FB45
:104EA00007F206FB07F70CFB06F616EB074642EB8C
:104EB000174205FB0CFC16EB0C4642EB1C456A182E
:104EC00054F1000148BF7047B619524141EB01014E
:104ED000A3F10103704795F0000F37D04FEA11425C
:104EE00021EA02464FEA144724EA074C02FB07F185
:104EF00006FB07F70CFB06F414EB074441EB1741E4
:104F000002FB0CFC14EB0C4441EB1C414FEA15472F
:104F100025EA074C02FB07F506FB07F70CFB06F634
:104F200016EB074645EB174502FB0CFC16EB0C464F
:104F300045EB1C42121951F1000148BF7047B619E8
:104F4000524141EB0101A3F1010370474FEA1445BF
:104F500024EA05464FEA114721EA074C05FB07F111
:104F600006FB07F70CFB06F212EB074241EB174179
:104F700005FB0CFC12EB0C4251EB1C414FF0000600
:104F800048BF7047921841EB0101A3F1010370473C
:104F9000490050EAC12018BF04204A0D18BF40F054
:104FA000010040F2FF72B2EB515F08BF40F0020017
:104FB000012808BF052070474100080218BF0420DF
:104FC0000A0E18BF40F001004FF07F4232EA0101A3
:104FD00008BF40F00200012808BF052070470121EA
:104FE00001F0F1BB0021084601F096B86FF05E01B8
:104FF000080701F0E8BB00002DE9F04D0D4614460E
:105000004FF07F41B1EB440F9EBF4FF0FF3129605D
:10501000BDE8F08D4FF0004040EA0421C4F3C750D2
:10502000783810F01F024A4B4FEA601CC2F120068C
:105030007B44C4F3C750A0F178004FEA601003EB43
:10504000800053F82C3008BFD0E901C612D0D0F848
:1050500004C093402CFA06F73B4387680CFA02FC25
:1050600027FA06F8C06807FA02F2F0404CEA080C8A
:1050700042EA0006A3FB0132ACFB01C0A6FB0161C2
:1050800001EB0C068E4234BF4FF0010C4FF0000CC8
:10509000C1186144BCF1000F02D0814202D903E083
:1050A000814201D2012000E00020104400F12002E2
:1050B0004FEA92188006CA0C40EA42304F03C5F806
:1050C000008001F03BF98246384601F04FF96FF05D
:1050D000120101F078FB0746304601F047F96FF006
:1050E000250101F070FB83463946504600F04CFF25
:1050F000594600F049FF00F500666FF30B06514674
:10510000304601F0B5FA394601F0B2FA594601F0DD
:10511000A5FA104901F0A6F907460F49304601F0FB
:10512000A1F9394600F030FF07460C49304601F03E
:1051300099F9394600F028FF14F0004F08BFBDE888
:10514000F08DC8F1805180F000402960BDE8F08DFD
:1051500054180000DB0FC92F22AAFD290000C92F17
:1051600030380A2801D20120704700207047000023
:105170002DE9F843044602464F486946B0EB420F1A
:1051800009D94FF0E640B0EB420F94BF00204FF03A
:10519000FF30009030E0494B22F00040834271D94B
:1051A0004749204601F05EF901F028FA804601F0F7
:1051B000A9F800F0030000904249404601F052F97E
:1051C00005464149404601F04DF906463F494046F3
:1051D00001F048F907463E49404601F043F92146AF
:1051E00001F03CFA394601F043FA314601F040FA49
:1051F000294601F03DFA04462546009C002C45DB7B
:10520000294614F0010F08461CD001F02BF9064680
:10521000304901F027F9304900F0B6FE314601F07F
:1052200021F92E4900F0B0FE314601F01BF9294664
:1052300001F018F9294600F0A7FE14F0020F1CD067
:10524000BDE8F88301F00EF90546254901F00AF999
:10525000244900F099FE294601F004F9224900F0A2
:1052600093FE294601F0FEF84FF07E5100F08CFECF
:1052700014F0020F08BFBDE8F88380F00040BDE8DD
:10528000F883FFE71046FFF7B7FEB4E76800B0F118
:105290007F4F3CBF4FF07E50BDE8F88307D14FF001
:1052A0000100FBF756F8BDE8F843FFF79BBE284620
:1052B000BDE8F843FFF793BEB61F927E490E4946FC
:1052C00083F9223F1A61342C0020A23300A0FD395B
:1052D0000000C93F336D4CB9DA82083CA0AA2ABE4F
:1052E000B93AB2BACA9F2A3DDDFFFFBE70B5054686
:1052F00001F084F904460146284601F0B9F915F099
:10530000004F4FF07F410ED0B0F13F4F28BFB1EBBF
:10531000400F0ED2B0F17C5F1DDDB1EB400F1AD310
:1053200013E0044617E0B0F13F4F08D9B1EB400F4E
:1053300005D34FF07E51204601F09AF9F1E7B0F124
:105340007C5F08DBB1EB400F05D34FF07E51204668
:1053500000F01AFEE5E7284664F31E0070BD000069
:105360002DE9F8430446024652486946B0EB420F25
:1053700009D94FF0E640B0EB420F94BF00204FF048
:10538000FF30009030E04C4B22F00040834271D956
:105390004A49204601F066F801F030F9804600F0F5
:1053A000B1FF00F0030000904549404601F05AF873
:1053B00005464449404601F055F8064642494046F4
:1053C00001F050F807464149404601F04BF82146AC
:1053D00001F044F9394601F04BF9314601F048F942
:1053E000294601F045F904462546009C002C45DB82
:1053F000294614F0010F08461ED001F033F8054687
:10540000334901F02FF8334900F0BEFD294601F081
:1054100029F8314900F0B8FD294601F023F84FF092
:105420007E5100F0B1FD14F0020F08BFBDE8F88313
:1054300080F00040BDE8F88301F014F806462749E3
:1054400001F010F8264900F09FFD314601F00AF8FE
:10545000244900F099FD314601F004F8294601F095
:1054600001F8294600F090FD14F0020FE0D1BDE8EC
:10547000F883FFE71046FFF7BFFDB4E76800B0F11F
:105480007F4F09D22846FFF797FD042808BFFFF792
:10549000ADFD2846BDE8F88306D10120FAF759FF93
:1054A000BDE8F843FFF79EBD2846BDE8F843FFF787
:1054B00096BD0000B61F927E490E494683F9223FF1
:1054C0001A61342C0020A23300A0FD390000C93F2E
:1054D000B93AB2BACA9F2A3DDDFFFFBE336D4CB95F
:1054E000DA82083CA0AA2ABE10B500290AD00878A2
:1054F000002807D005487844FBF74CFF002801D06E
:10550000002010BD0248784410BD0000721E00004B
:105510006A1E000010B500290AD00878002807D0BC
:1055200005487844FBF736FF002801D0002010BD65
:105530000248784410BD0000621E00005A1E0000A0
:1055400021F0004201F00043A2F16052B2F5801F49
:1055500028BFD2F17F6C0BD95FEA001C43EAC2027C
:1055600042EB507018BF704728BF20F00100704711
:10557000B2F5801FBCBF184670474FEA410C1CF5BE
:10558000001F02D2084601F034B870B500F08EFB5F
:1055900000000089FFF7F6BF4FF00040A0F5800043
:1055A0007047000010B591EA030F48BF83F0004335
:1055B00000F1D883841A71EB030C05D2121943EB66
:1055C0000C03001B61EB0C014FEA1154A4EB135CBC
:1055D000DFF81CE11EEA430F18BF9EEA445F00F0AB
:1055E000748021EA045123EA0E0343F48013DCF1B2
:1055F000200E32D322FA0CFE10EB0E0023FA0CFE22
:1056000041EB0E01CCF1200E03FA0EFE10EB0E0062
:10561000CCF1200E51F10001B1F5801F32D201EB27
:10562000045112FA0EF2BDE8104058BF7047401CFA
:1056300038BF5FEA420218BF7047002814BF20F04D
:10564000010041F100014FEA410313F5001F38BF8B
:105650007047A1F1C04100F077BB012A43EB030280
:10566000ACF1200CDCF11F0E32BF4FF0000E23FA1C
:105670000CF310EB030041EB0451B4EB115FD0D0FD
:10568000A1EB045101F58011490801EB04515FEAD7
:1056900030000ED350F1000038BF12FA0EFE08D1D0
:1056A000BDE81040C9E7401C38BF5FEA4202CAD1DA
:1056B000C3E7BDE810404FEA410313F5001F38BFB0
:1056C0007047A1F1C04100F03FBB9EEA445F08D0A3
:1056D00011EA5E0FBDE8104004BF01F00041002058
:1056E0007047BDE8104070B500F0E0FA64FBBE3EC4
:1056F0000000E0FF491058BFC1F140415B1058BFA6
:10570000C3F140438B42EFF3008070472DE9C04165
:1057100030B4DFF8A4C23CEA111418BF3CEA1314F9
:1057200000F0ED801CEA111481EA030544EAD57407
:1057300018BF1CEA131500F0C880A4EB050404F19F
:105740007F7404F500344FF0004545EAC12145EA75
:10575000C32341EA505143EA52534FEAC0204FEA73
:10576000C222994208BF904200F09D804FEA136523
:105770000FF24416765D4FEA134506FB05F7C7F1B5
:10578000807706FB07F74FEAD737A7FB0368764217
:10579000A7FB06CEC8F5803838BFA8F1010807FB83
:1057A00008E6A6FB028C4FF0000EE6FB03CEDCF110
:1057B000000CCEF1004E38BFAEF1010EA6FB0C5826
:1057C0004FF00007E6FB0E87A1FB08C6A0FB07CE43
:1057D00016EB0E064FF0000545F10005E1FB0765ED
:1057E00015F1E04E7EBFA4F580345FEA46066D41B8
:1057F00016F1800745F100054FEA172747EA0567CC
:105800004FEA15254FEA0666A6F1DE46B6F1805F3F
:1058100020D9384605EBC47124F0010C01EB0C11C2
:10582000BCF1FE6F02D8F0BCBDE8008124425CBF31
:1058300001F5801E9EEAC47F02D4F0BCBDE8008161
:10584000244200F13980A1F1C041F0BCBDE8004123
:1058500000F07ABA4FEAD02040EA41504FEAD12115
:105860004FEAD22242EA43524FEAD323A7FB0286F1
:1058700007FB036605FB02661EEA0E0F58BFA6EB88
:105880000056B6EB00564FEA520E4EEAC37E18EBB6
:105890000E0E56EB530EBCD518EB02085E417F1C72
:1058A00055F10005B5E74FF480154FF000074FF0B4
:1058B00000064FF00008ACE701F1C04101F00041E3
:1058C0004FF00000F0BCBDE800810CEA131511EAAE
:1058D0000C1F00D00CE013EA0C1F00F026804FF0E4
:1058E000000081EA030101F00041F0BCBDE8008145
:1058F000F0BCBDE8004181EA030100F025BAF0BC2C
:10590000BDE8004170B500F0D1F900BF097EFC3E52
:1059100000F007B84FF0000081EA030101F00041F8
:10592000704781EA030100F00FBAF0BCBDE8004106
:1059300022494FF000007047FFFDFBF9F7F5F4F244
:10594000F0EEEDEBE9E8E6E4E3E1E0DEDDDBDAD81A
:10595000D7D5D4D3D1D0CFCDCCCBCAC8C7C6C5C478
:10596000C2C1C0BFBEBDBCBBBAB9B8B7B6B5B4B38F
:10597000B2B1B0AFAEADACABAAA9A8A8A7A6A5A47A
:10598000A3A3A2A1A09F9F9E9D9C9C9B9A9999983E
:105990009797969595949393929191908F8F8E8EE1
:1059A0008D8C8C8B8B8A898988888787868585846E
:1059B00084838382828181800000FF070000F87F5A
:1059C00051EA030C17D41CF5801F58BFBCF5801F8B
:1059D00000F10680994218BF704708BF9042704797
:1059E00007D711F5801F58BF13F5801F19D49942AE
:1059F0007047894270471CF5801F08D5BCF5801F91
:105A0000F7D58B4218BF704708BF824270474FF4EA
:105A1000001C1CEB410F38BF1CEB430F01D28B4223
:105A2000704770B500F042F9922449004FF00051E0
:105A30004FF08053FFF75EBE10F0004248BF404277
:105A4000B0FA80F310FA03F10AD0C3F11D0303F595
:105A5000806302EB03524FEA415002EBD1217047C1
:105A60004FF000007047000051EA030C17D41CF5FA
:105A7000801F58BFBCF5801F00F10680994218BFF7
:105A8000704708BF9042704707D711F5801F58BF75
:105A900013F5801F19D499427047894270471CF54D
:105AA000801F08D5BCF5801FF7D58B4218BF704703
:105AB00008BF824270474FF4001C1CEB410F38BFF7
:105AC0001CEB430F01D28B42704770B500F0EEF82B
:105AD000922449004FF080514FF00053FFF70ABE67
:105AE00051EA030C17D41CF5801F58BFBCF5801F6A
:105AF00000F10680994218BF704708BF9042704776
:105B000007D711F5801F58BF13F5801F19D499428C
:105B10007047894270471CF5801F08D5BCF5801F6F
:105B2000F7D58B4218BF704708BF824270474FF4C9
:105B3000001C1CEB410F38BF1CEB430F01D28B4202
:105B4000704770B500F0B2F8922449004FF0005150
:105B50004FF08053FFF7CEBD70B5DFF848C11CEAA7
:105B6000111E1EBF1CEA13159EEA0C0F95EA0C0FBE
:105B700000F06F8081EA03044EEAD47EAE4421EA4D
:105B80004C1123EA4C1341F4801143F48013AEF11D
:105B90007F7EA1FB024CA0FB0365361955EB0C057B
:105BA000A1FB034C4CF10003A0FB021C16EB0C06FE
:105BB000654153F10003094218BF46F0010613F492
:105BC000007F0BD14FEA03314FEA053041EA15510E
:105BD00040EA165034036FF003020AE04FEAC32193
:105BE0004FEAC52041EA555140EA5650F4026FF0A1
:105BF000020202EB2E4201EB025585EACE710AD079
:105C00005FEA440C18BF24F0004450F1000041F159
:105C1000000120EAD47040F2FE7C624500D270BDE3
:105C2000A84214BF4FF080444FF04044002E08BFFC
:105C30000024BEF1806FA8BFA1F1C041BDE8704053
:105C400080F2828001F1C04101F000414FF000007C
:105C500070470CEA13159EEA0C0F18BF95EA0C0F5B
:105C600006D081EA030E4FF000000EF0004170BD37
:105C700000F01CF88900013E00F007B800F009B8F8
:105C80004FEA430C5FEA5C5C08D081EA030100F054
:105C90005BB84FEA410C5FEA5C5CF6D102494FF019
:105CA000000070470000FF070000F87F0EF1020EB1
:105CB0002EF0030E5EF8046B364205D4012A43EB46
:105CC000030515F5001F12D8012841EB010C1CF546
:105CD000001F0CD80ED14FEAD17C0CEB4C0C0CF110
:105CE000020C15F5001F08BF4CEBD37C04E04FF00D
:105CF000080C01E04FEAD37C0CEB4C0526FA05F6C4
:105D000006F00706B6F1040C06D20EEB860CBDE8D1
:105D100070404CF0010C6047DFE80CF0090B020208
:105D20004FF00041A1F500214FF0000070BD194671
:105D30001046012851EB010418BFD4F5001484BFAC
:105D4000002001F0004170BD0808A0F500114FEAE5
:105D50003101704710B591EA030F48BF83F000434B
:105D60003FF528AC841A71EB030C07D28CF0004C81
:105D7000121943EB0C03001B61EB0C014FEA1154A9
:105D8000A4EB135CDFF8A4E11EEA430F18BF9EEA00
:105D9000445F00F0B48021EA045123EA6E035242CA
:105DA000C3EB6E0338BF5B1EDCF1200E25D322FA55
:105DB0000CFE10EB0E0043FA0CFE41EB0E01CCF191
:105DC000200E03FA0EFE10EB0E00CCF1200E51F166
:105DD000000129D401EB045112FA0EF2BDE8104083
:105DE00058BF7047401C1CBFB2F1004F70470028DD
:105DF0000CBF491C20F00100704712EB020E43EB70
:105E0000030218BF4FF0010E4EEA4202ACF1200C23
:105E1000DCF11E0E56D943FA0CFE10EB0E00CCF14D
:105E20001E0E51F1FF31D5D50EF1010E12FA0EFE04
:105E3000404141EB010101EB445C5FEA5C5C10D93D
:105E400001EB045110EBDE7038BFBEF1004FBDE82E
:105E5000104018BF704700280CBF491C20F00100FB
:105E6000704734D24FEAD42C24F4006411F50011A9
:105E70001BD0B1FA81F20B3AA41AA41ED2F120036E
:105E8000914030FA03F31943904001EBCC7101EBE0
:105E90000451002CBDE81040A8BF704701F1C0417B
:105EA00001F000414FF000007047B0FA80F310FAA3
:105EB00003F102D1BDE810407047E41A173C4805D1
:105EC000C90AE2E701EB0451BDE8104070474910F0
:105ED0004FEA300001EB0451BDE8104002E04FF002
:105EE000000170474A0008BF0042F8D0B2F5001F19
:105EF00028BF704701F000414FF0000070479EEA54
:105F0000445F07D011EA5E0FBDE8104004BF0021D6
:105F100000207047BDE8104070B5FFF7C7FE00BF16
:105F200040DFF63E104683F0004170470000E0FF7E
:105F300043004FEAD30C4FEA3C0C43401FBF4007DD
:105F40000CF1605113F0FE4F70471CF0006F03D14D
:105F50000CF00041002070470CF0004343EA507001
:105F600040EACC0010B500F0FEFA00BF000000923D
:105F70004FEA0001FFF7E8BE4FF00041A1F5002114
:105F80004FF000007047000090EA010F48BF81F019
:105F9000004100F17483421A3CBF801A89184FEA0D
:105FA000D052A2EBD1534FF07F4C1CEA410F18BFE7
:105FB0009CEA026F00F03B804FF0004C4CEA00205E
:105FC0004CEA012121FA03FC10EB0C0C1ED202F169
:105FD000FF325FEA1C2040EBC25038BF70471CF014
:105FE0007F0F4FEA400C18BFBCF17F4F38BF70479E
:105FF000C3F12003994008BF20F00100BCF17F4F9E
:1060000038BF7047A0F1C04000F0F3BA4FEA3C003F
:10601000000A40EBC25028BF1CF0FF0F4FEA400CB3
:10602000E6D018BFBCF17F4F38BF7047EAE79CEA63
:10603000026F05D010EA5C0F08BF00F00040704707
:1060400010B500F090FA00BF64FBBE3E014800F0BE
:1060500088BB00BF0000C07F10B5FFF7B1FC0CBFCC
:106060000120002010BD10B5FFF7AAFC14BF0120CD
:10607000002010BD10B5FFF7F7FC8CBF01200020F9
:1060800010BD10B5FFF7F0FC2CBF0120002010BDA3
:1060900010B5FFF725FD94BF0120002010BD10B5FD
:1060A000FFF71EFD34BF0120002010BD10B500F029
:1060B000F5F80CBF0120002010BD10B500F0EEF87F
:1060C00014BF0120002010BD10B500F063F98CBF93
:1060D0000120002010BD10B500F05CF92CBF01209C
:1060E000002010BD10B500F089F994BF01200020F8
:1060F00010BD10B500F082F934BF0120002010BDA2
:10610000401058BFC0F14040491058BFC1F1404154
:106110008142EFF3008070474FF47F0C1CEAD012ED
:106120001EBF1CEAD11392EA0C0F93EA0C0F00F089
:10613000858090EA010F48BF42F4807240F4000C61
:1061400041F400002CF07F4120F07F4000B5A2EB2D
:10615000030281420FF2081CACEB504E9EF800E0A7
:10616000C0F100004FEA4E0E00FB0EFC38BF4900A4
:106170004FEA2C1C0CFB0EF34FEACE1E0EEB635EB7
:106180004FEA112C0EFB0CFC4FEAC1214FEA1C53C5
:1061900000FB031102F5FA024FEA112C0EFB0CFC76
:1061A0004FEA01314FEADC4C00FB0C1142EB22427A
:1061B000C14228BF09184CEB03335DF804EB10EB28
:1061C000410143EBC250B2F57C0F38BF704729D56F
:1061D00012F0F00F1CBF00F1C04000F0004070470B
:1061E000008182838485868788898B8C8D8E8F91B0
:1061F0009293959697999A9C9D9FA0A2A3A5A7A8D4
:10620000AAACAEB0B2B3B5B7B9BCBEC0C2C5C7C9FF
:10621000CCCED1D4D7D9DCDFE2E6E9ECF0F3F7FA63
:10622000FE0000004FEA400C0CF1807CBCF17E4F78
:1062300028BF7047B0F1C04000F0DBB90CEAD113C1
:1062400090EA010F48BF42F48072624538BF63454F
:1062500007D213F47F0F16D080EA010000F000404F
:10626000704710B500F07FF9097EFC3E00F005B8DC
:1062700080EA010000F00040704780EA010000F071
:10628000004000F0B6B912F47F0F04BF0248704717
:1062900080EA010000F0ADB90000C07F50EA010CB7
:1062A00000F113801CF5000F58BFBCF5000F01D49E
:1062B0008842704707D710F5000F58BF11F5000F3F
:1062C00015D488427047894270471CF5000F04D5E9
:1062D000BCF5000FF7D5814270474FF0807C1CEB76
:1062E000400F38BF1CEB410F01D28142704710B5FF
:1062F00000F039F9922449004FF000504FF08051DE
:10630000FFF7FEBE41000B0ED3F19E0208D950F4F8
:1063100000034FEA032323FA02F048BF40427047CC
:1063200010B500F020F900BF49922480002070478A
:106330006FF0004282EA20007047000010F0004138
:1063400048BF4042B0FA80F310FA03F2C3F19D0354
:106350000BD051EAC35101EB1220530638BF7047EE
:1063600000F1010008BF20F001007047B0FA80F38F
:1063700010FA03F2C3F19D030AD0D90501EB1220F4
:10638000530638BF704700F1010008BF20F001003C
:106390007047000050EA010C00F113801CF5000F5B
:1063A00058BFBCF5000F01D48842704707D710F5DD
:1063B000000F58BF11F5000F15D48842704789426D
:1063C00070471CF5000F04D5BCF5000FF7D58142CE
:1063D00070474FF0807C1CEB400F38BF1CEB410F27
:1063E00001D28142704710B500F0BDF892244900F7
:1063F0004FF080504FF00051FFF782BE50EA010C81
:1064000000F113801CF5000F58BFBCF5000F01D43C
:106410008842704707D710F5000F58BF11F5000FDD
:1064200015D488427047894270471CF5000F04D587
:10643000BCF5000FF7D5814270474FF0807C1CEB14
:10644000400F38BF1CEB410F01D28142704710B59D
:1064500000F089F8922449004FF000504FF080512D
:10646000FFF74EBE4FF47F0C1CEAD0121EBF1CEA91
:10647000D11392EA0C0F93EA0C0F00F0478090EAD8
:10648000010F48BF42F480724FF0004C4CEA0020EC
:106490004CEA012102EB0302A0FB0113A2F500026A
:1064A000002918BF43F001035B0028BF4FEA330304
:1064B00042EB22425FEA132C4CEBC2502EBFBCEBE6
:1064C000436FB2F57C0F70474FEA036CBCF1004F8D
:1064D00008BF20F00100B2F57C0F38BF70470BD524
:1064E00082F0FF0212F5803FC8BF704700F1C04044
:1064F000D8BF00F00040704700F5000C5FEA4C0C7C
:1065000048BF7047B0F1C04000F073B80CEAD11337
:1065100090EA010F48BF42F48072624538BF63457C
:1065200004D280EA010000F00040704710B500F08E
:106530001AF800BF8900013E00F007B800F009B862
:106540005FEA410C5FEA1C6C08D080EA010000F0B1
:1065500050B85FEA400C5FEA1C6CF6D14FF0004087
:10656000A0F5800070470EF1020E2EF0030E5EF8CB
:10657000044B244204D44FEA4102B2F17F4F11D8B8
:106580004FEA4003B3F17F4F0CD80ED14FEAD07CD5
:106590000CEB4C0C0CF1020CB2F17F4F08BF4CEB32
:1065A000D17C04E04FF0080C01E04FEAD17C0CEB09
:1065B0004C0324FA03F404F00704B4F1040C06D2EB
:1065C0000EEB840CBDE810404CF0010C6047DFE896
:1065D0000CF0070802024FF00040A0F5800010BD4B
:1065E0000846420018BFD2F1807288BF00F0004018
:1065F00010BDFF2141EAD050C00570475FEA400C52
:106600005FEA1C6CBCF17F0314D4D3F1170240F392
:106610001C804FF0010C0CFA02FCACF101030340AA
:1066200020EA0300B3EB5C0208BF10EA0C0F88BF3E
:1066300060447047B3F1FF3F28BF5FEA002C00F0D1
:10664000004088BF40F07E507047BCF1FF0FB8BFDC
:10665000704710B5FFF787FF40DBB6BE80F0004003
:1066600090EA010F7FF597AC81F0004100F007B888
:1066700090EA010F48BF81F000413FF58CAC421A0F
:1066800004D882F00042A0EB020011444FEAD0523D
:10669000A2EBD1534FF07F4C1CEA410F18BF9CEA8C
:1066A000026F4AD04FF0004C4CEA00204CEA012126
:1066B00021FA03FCB0EB0C0C0FD412F0FE0F36D015
:1066C0005FEA4C001DD5001240EBC25038BF704746
:1066D0001CF03F0F18BF70470BE05FEA1C20A2F1CF
:1066E000010240EBC25038BF70471CF07F0F18BF4B
:1066F0007047C3F12003994014BF401E20F00100F1
:1067000070474FEA1223800808BF7047B0FA80FC38
:10671000A2EB0C02CCF1280C60FA0CF093EA122FD9
:1067200004BF00EBC25070474FEAC3707047130AB2
:106730005FEADC1008BF7047F6E79CEA026F04D0FE
:1067400010EA5C0F08BF0020704710B5FFF70BFF81
:1067500040DFF63E81F000407047FAF729BAFAF7B9
:106760005DBB0CF00F03092B08BF082000F051801F
:106770000A2B0BD0082B18BF704708BF1CF0400F26
:106780000AD04FF000004FF0000170471CF0400F9E
:1067900018BF4FF0004070471CF0100F08D000F0F9
:1067A0007F4220F0704342EAD3014FEA43707047C2
:1067B00000F0604021F07F4242EA000201F07F4099
:1067C00040EA727070474FF0FF0212EAD0521CBFCD
:1067D00092F0FF038B42C2BFD14200EBC150704721
:1067E000002A0AD0002B0BD000F000400029A4BFE3
:1067F00040F0FE4040F40000704700F00040704759
:1068000043024FF00B0C18BF4CF0806C7FF41EACB1
:1068100070471CF4801F11D01CF4E02F03D06FEAE6
:10682000CC31490070474FF04050EFF3008222F026
:10683000704242EA000282F3008870474FF0000085
:1068400070470000000000000000000030313233CB
:106850003435363738394142434445464030580094
:1068600030313233343536373839616263646566C6
:106870004030780004000008000000000000000222
:106880000001000010000000000000006E83F9A26B
:106890002915444ED15727FCC0DD34F5999562DBAC
:1068A0004190433CAB6351FE30313233343536379F
:1068B0003839616263646566787000303132333430
:1068C0003536373839414243444546585000000078
:1068D00002400000000000A0000000000540000091
:1068E000000000C8000000000C4000000000409CB8
:1068F00000000000194000000020BCBE00000000A5
:1069000034400000BFC91B8E00000004B5400000E9
:10691000504BCFD06607E2CF010000006C41000071
:106920003E8251AADFEEA73401000000D9420000E8
:10693000DCB5A0E23A301F97FFFFFFFFB44500002F
:10694000FD25A0C8E9A3C14FFFFFFFFFFF3F0000E7
:106950000000008000000000FF3F000000000080F9
:10696000000000000000000000000000010203041D
:1069700006070809000000000102030402030405E1
:10698000060708090A0B0C0D0E0F10100102050076
:1069900000000000000000000002004040404040B5
:1069A000400040000450505000000000000000086B
:1069B000000A0A3F14147E2828000610103C50508C
:1069C0003814147810080030494A3408162949064A
:1069D0000800304848324A444639000240404000EE
:1069E0000000000000000400102040404040402013
:1069F00010040040201010101010204006105438D1
:106A0000541000000000000800000808087F080873
:106A10000800030000000000000020202004000007
:106A200000000070000000000200000000000000F4
:106A300040400004000010102020204040000600CC
:106A4000384444444444443800040020602020205A
:106A5000202070000600384404081020407C000606
:106A60000038440418040444380006000818284874
:106A70007C0808080006007C404078040444380084
:106A8000060018204078444444380006007C04087E
:106A9000081010202000060038444438444444388C
:106AA000000600384444443C040830000200000062
:106AB0004040000040400003000000202000002073
:106AC0002020070000020C3040300C0200080000BB
:106AD00000007F007F00000007000040300C020C27
:106AE0003040000500700808102020002000083EFB
:106AF000419DA5A5A59F403C00070018182424240B
:106B00007E424200060078444478444444780007BA
:106B1000001E2040404040201E00070078444242B2
:106B2000424244780006007C4040784040407C006F
:106B300006007C40407C404040400007001E204052
:106B4000404E42221E0007004242427E42424242E2
:106B5000000400702020202020207000050038084C
:106B60000808080808700006004448506060504853
:106B70004400050040404040404040780008006329
:106B800063555549494141000700626252524A4AE1
:106B900046460008001C2241414141221C000600DB
:106BA00078444444784040400008001C2241414160
:106BB00041221C04070078444444784844420006BB
:106BC000003C404038040404780006007C1010109B
:106BD00010101010000700424242424242423C0064
:106BE0000600444444282828101000080049494958
:106BF0003636361212000600444428101028444449
:106C000000060044442828101010100006007C04E0
:106C100008101020407C000470404040404040403C
:106C2000700004004040202020201010000470104C
:106C300010101010101070000800081422410000FD
:106C4000000000070000000000000000007E03407C
:106C50002000000000000000000600000038043C96
:106C600044443C0006404040784444444478000595
:106C700000000038404040403800060404043C4412
:106C80004444443C000600000038447C4044380042
:106C90000430404070404040404000060000003C4E
:106CA000444444443C040640404078444444444402
:106CB00000020040004040404040400003002000EF
:106CC000602020202020200640404048506050484E
:106CD0004400020040404040404040400008000066
:106CE0000076494949494900060000007844444477
:106CF0004444000600000038444444443800060080
:106D0000000078444444447840060000003C444479
:106D100044443C04040000005060404040400005F2
:106D200000000038406018087000040040407040C7
:106D300040404030000600000044444444443C00CD
:106D400006000000444428281010000800000049F4
:106D500049555522220006000000442810102844FE
:106D60000006000000444428281010200500000000
:106D70007808102040780004102020204040202077
:106D800020100240404040404040404040044020ED
:106D9000202010102020204008000000003149462B
:106DA0000000000400705050505050507000080017
:106DB0007E10101E111111120006007C4040404050
:106DC000404040000300000000000000202040057B
:106DD00008100078404040404000050000000000DE
:106DE00000002828500800000000000000004900B2
:106DF0000610107C101010101000000610107C10EF
:106E0000107C1010000007001C2278207820120C43
:106E10000007609090621CE0629494620800382839
:106E200028282E29294E00040000001020402010A0
:106E3000000008004848487E4949494E000700467E
:106E4000484870504844420008007E10101E11113E
:106E5000111100070042424242427E08080007200A
:106E600078203C22222222220403404020000000FD
:106E7000000000000320204000000000000000058A
:106E80005050280000000000000005282850000095
:106E9000000000000005000000003078783000009D
:106EA0000700000000007E00000000080000000055
:106EB00000FF0000000005000000000000000000CE
:106EC000000700EA4E4A4A000000000008000000E7
:106ED00078484E49498E00040000004020102040B0
:106EE00000000800000048487E49494E000608108E
:106EF000004C506050484400072078203C22222259
:106F0000222200060000004444447C1010000500CA
:106F1000000000000000000000050000000000006C
:106F20000000000005000000000000000000000557
:106F300000380808080808087000060000004438F7
:106F4000283844000006047C404040404040400057
:106F50000200404040000040404000063C404038B5
:106F600044443804047806007C4040784040407C2B
:106F70000008003C4299A1A1A199423C06001C20B6
:106F800040784040201C00060000001428502814BF
:106F900000000700000000007E0202020004000062
:106FA000000000700000000008003C42999599958F
:106FB00095423C04500070202020202020700500C5
:106FC00030484830000000000006000010107C101F
:106FD00010007C000400702020202020207000027F
:106FE0000040004040404040400005000808784014
:106FF00040404040000600444444444C744040003B
:1070000006003C7474743414141400020000004030
:107010004000000000000600280038447C4044384E
:107020000008008ACDCAA8AF989888000500000023
:1070300038407040403800060000005028142850A6
:107040000000032000602020202040000006003CBB
:1070500040403804040478000500000038406018FF
:10706000087000040050002020202020200007008D
:1070700018182424247E42420006007C40407844B4
:107080004444780006007844447844444478000638
:10709000007C404040404040400008000E0A121270
:1070A000127F41410006007C4040784040407C0017
:1070B000080049492A2A1C2A4908000600780404C5
:1070C000380404047800070042464A4A5252624299
:1070D0000007241842464A4A5262420007004648C6
:1070E0004870504844420007003E222222222222B9
:1070F0004200080063635555494941410007004279
:1071000042427E424242420008001C22414141412B
:10711000221C0007007E42424242424242000600D8
:1071200078444444784040400007001E20404040DE
:1071300040201E0006007C101010101010100007D8
:10714000004242242418181060000800083E4949F3
:1071500049493E08000600444428101028444400D1
:10716000080042424242427F01010007004242427F
:10717000423E020202000800494949494949497F03
:1071800000080049494949494949FF8008007010F1
:10719000101E1111111E000800414141794545455D
:1071A0007900060040404078444444780007007865
:1071B00004023E020204780008004E515171515100
:1071C000514E0007001E2222221E122242000600FB
:1071D000000038043C44443C00061C2040784444F1
:1071E00044443800060000007844784444780005A0
:1071F000000000784040404040000700001C14148C
:1072000024247E42000600000038447C40443800BC
:1072100008000000492A2A1C2A49000500000070C5
:1072200008300808700006000000444C54644444D0
:107230000006241800444C54644444000600000036
:107240004C506050484400060000003C2424242494
:10725000440006000000446C5454444400060000FE
:107260000044447C44444400060000003844444444
:10727000443800060000007C4444444444000600B6
:107280000000784444784040000500000038404049
:1072900040403800060000007C101010101000065E
:1072A00000000044442828101020080808083E491F
:1072B0004949493E080600000044281010284400AF
:1072C0000600000048484848487C04060000004486
:1072D00044443C0404000800000049494949497FEE
:1072E00000080000004949494949FF8007000000A3
:1072F00070101C12121C0008000000414179454525
:107300007900060000004040784444780005000001
:107310000070083808087000080000008E91F19194
:10732000918E00060000003C44443C244400486127
:1073300072727920506F74746572205468656D653F
:107340000078252E316600009874000800000020A7
:107350001000000028010008A87400081000002098
:10736000C8090000440100081C00000043000000A0
:10737000F8FFFFFF0C0000000E0000000F000000EF
:107380002E0000001001000043000000F8FFFFFF86
:107390000040404040404040404041414141414028
:1073A00040404040404040404040404040404040DD
:1073B000400502020202020202020202020202026C
:1073C0000220202020202020202020020202020271
:1073D00002029090909090901010101010101010C9
:1073E00010101010101010101010101002020202D5
:1073F0000202888888888888080808080808080819
:107400000808080808080808080808080202020214
:10741000400000000000000000000000000000002C
:10742000000000000000000000000000000000005C
:10743000000000000000000000000000000000004C
:10744000000000000000000000000000000000003C
:10745000000000000000000000000000000000002C
:10746000000000000000000000000000000000001C
:10747000000000000000000000000000000000000C
:1074800000000000000000000000000000000000FC
:10749000000000000000000000127A0000002041FF
:0874A0000100000010000000D3
:04000005080000ED02
:00000001FF
